Component: ARM Compiler 5.05 update 1 (build 106) Tool: armlink [4d0efa]

==============================================================================

Section Cross References

    app.o(.text) refers to os_q.o(.text) for OSQCreate
    app.o(.text) refers to os_mem.o(.text) for OSMemCreate
    app.o(.text) refers to os_time.o(.text) for OSTimeDlyHMSM
    app.o(.text) refers to bsp_key.o(.text) for bsp_KeyScan
    app.o(.text) refers to stm32f2xx_gpio.o(.text) for GPIO_ResetBits
    app.o(.text) refers to os_task.o(.text) for OSTaskCreate
    app.o(.text) refers to bsp.o(.text) for bsp_Init
    app.o(.text) refers to cpu_core.o(.text) for CPU_Init
    app.o(.text) refers to lib_mem.o(.text) for Mem_Init
    app.o(.text) refers to bsp_int.o(.text) for BSP_IntDisAll
    app.o(.text) refers to os_core.o(.text) for OSInit
    app.o(.text) refers to app.o(.bss) for RPM_Q
    app.o(.text) refers to app.o(.data) for counter
    os_app_hooks.o(.text) refers to cpu_a.o(.text) for CPU_SR_Save
    os_app_hooks.o(.text) refers to os_var.o(.data) for OS_AppTaskCreateHookPtr
    bsp.o(.text) refers to misc.o(.text) for NVIC_PriorityGroupConfig
    bsp.o(.text) refers to bsp_led.o(.text) for bsp_InitLed
    bsp.o(.text) refers to bsp_key.o(.text) for bsp_InitKey
    bsp.o(.text) refers to stm32f2xx_rcc.o(.text) for RCC_GetClocksFreq
    bsp.o(.text) refers to os_cpu_c.o(.text) for OS_CPU_SysTickInit
    bsp.o(.text) refers to cpu_core.o(.text) for CPU_TS_TmrFreqSet
    bsp.o(.text) refers to uldiv.o(.text) for __aeabi_uldivmod
    bsp.o(.text) refers to os_cfg_app.o(.constdata) for OSCfg_TickRate_Hz
    bsp_led.o(.text) refers to stm32f2xx_rcc.o(.text) for RCC_AHB1PeriphClockCmd
    bsp_led.o(.text) refers to stm32f2xx_gpio.o(.text) for GPIO_Init
    stm32f2xx_it.o(.text) refers to stm32f2xx_usart.o(.text) for USART_GetITStatus
    bsp_key.o(.text) refers to stm32f2xx_rcc.o(.text) for RCC_AHB1PeriphClockCmd
    bsp_key.o(.text) refers to stm32f2xx_gpio.o(.text) for GPIO_Init
    bsp_key.o(.text) refers to bsp_key.o(.bss) for s_tKey
    bsp_key.o(.text) refers to bsp_key.o(.data) for ret
    bsp_int.o(.text) refers to cpu_c.o(.text) for CPU_IntSrcDis
    bsp_int.o(.text) refers to cpu_a.o(.text) for CPU_IntDis
    bsp_int.o(.text) refers to os_core.o(.text) for OSIntEnter
    bsp_int.o(.text) refers to bsp_int.o(.bss) for BSP_IntVectTbl
    startup_stm32f2xx.o(RESET) refers to startup_stm32f2xx.o(STACK) for __initial_sp
    startup_stm32f2xx.o(RESET) refers to startup_stm32f2xx.o(.text) for Reset_Handler
    startup_stm32f2xx.o(RESET) refers to stm32f2xx_it.o(.text) for NMI_Handler
    startup_stm32f2xx.o(RESET) refers to os_cpu_a.o(CODE) for OS_CPU_PendSVHandler
    startup_stm32f2xx.o(RESET) refers to os_cpu_c.o(.text) for OS_CPU_SysTickHandler
    startup_stm32f2xx.o(.text) refers to system_stm32f2xx.o(.text) for SystemInit
    startup_stm32f2xx.o(.text) refers to entry.o(.ARM.Collect$$$$00000000) for __main
    stm32f2xx_adc.o(.text) refers to stm32f2xx_rcc.o(.text) for RCC_APB2PeriphResetCmd
    stm32f2xx_dac.o(.text) refers to stm32f2xx_rcc.o(.text) for RCC_APB1PeriphResetCmd
    stm32f2xx_gpio.o(.text) refers to stm32f2xx_rcc.o(.text) for RCC_AHB1PeriphResetCmd
    stm32f2xx_i2c.o(.text) refers to stm32f2xx_rcc.o(.text) for RCC_APB1PeriphResetCmd
    stm32f2xx_rcc.o(.text) refers to stm32f2xx_rcc.o(.data) for APBAHBPrescTable
    stm32f2xx_tim.o(.text) refers to stm32f2xx_rcc.o(.text) for RCC_APB2PeriphResetCmd
    stm32f2xx_usart.o(.text) refers to stm32f2xx_rcc.o(.text) for RCC_APB2PeriphResetCmd
    stm32f2xx_syscfg.o(.text) refers to stm32f2xx_rcc.o(.text) for RCC_APB2PeriphResetCmd
    system_stm32f2xx.o(.text) refers to system_stm32f2xx.o(.data) for SystemCoreClock
    cpu_core.o(.text) refers to cpu_a.o(.text) for CPU_SR_Save
    cpu_core.o(.text) refers to lib_mem.o(.text) for Mem_Clr
    cpu_core.o(.text) refers to bsp.o(.text) for CPU_TS_TmrInit
    cpu_core.o(.text) refers to lib_str.o(.text) for Str_Copy_N
    cpu_core.o(.text) refers to cpu_core.o(.bss) for CPU_Name
    cpu_core.o(.text) refers to cpu_core.o(.data) for CPU_TS_TmrFreq_Hz
    cpu_core.o(.text) refers to cpu_core.o(.constdata) for CPU_CntLeadZerosTbl
    cpu_c.o(.text) refers to cpu_a.o(.text) for CPU_SR_Save
    lib_math.o(.text) refers to cpu_a.o(.text) for CPU_SR_Save
    lib_math.o(.text) refers to lib_math.o(.data) for Math_RandSeedCur
    lib_mem.o(.text) refers to lib_mem_a.o(.text) for Mem_Copy
    lib_mem.o(.text) refers to cpu_core.o(.text) for CPU_SW_Exception
    lib_mem.o(.text) refers to cpu_a.o(.text) for CPU_SR_Save
    lib_mem.o(.text) refers to lib_mem.o(.bss) for Mem_PoolHeap
    lib_mem.o(.text) refers to lib_mem.o(.data) for Mem_PoolTbl
    lib_str.o(.text) refers to lib_ascii.o(.text) for ASCII_ToLower
    lib_str.o(.text) refers to lib_str.o(.constdata) for Str_MultOvfThTbl_Int32U
    os_cfg_app.o(.constdata) refers to os_cfg_app.o(.bss) for OSCfg_IdleTaskStk
    os_core.o(.text) refers to cpu_a.o(.text) for CPU_SR_Save
    os_core.o(.text) refers to os_cpu_c.o(.text) for OSIdleTaskHook
    os_core.o(.text) refers to os_task.o(.text) for OSTaskCreate
    os_core.o(.text) refers to os_prio.o(.text) for OS_PrioInit
    os_core.o(.text) refers to os_flag.o(.text) for OS_FlagInit
    os_core.o(.text) refers to os_mem.o(.text) for OS_MemInit
    os_core.o(.text) refers to os_msg.o(.text) for OS_MsgPoolInit
    os_core.o(.text) refers to os_mutex.o(.text) for OS_MutexInit
    os_core.o(.text) refers to os_q.o(.text) for OS_QInit
    os_core.o(.text) refers to os_sem.o(.text) for OS_SemInit
    os_core.o(.text) refers to os_tick.o(.text) for OS_TickTaskInit
    os_core.o(.text) refers to os_tmr.o(.text) for OS_TmrInit
    os_core.o(.text) refers to os_dbg.o(.text) for OS_Dbg_Init
    os_core.o(.text) refers to os_cfg_app.o(.text) for OSCfg_Init
    os_core.o(.text) refers to os_cpu_a.o(CODE) for OSIntCtxSw
    os_core.o(.text) refers to bsp.o(.text) for CPU_TS_TmrRd
    os_core.o(.text) refers to os_var.o(.data) for OSIdleTaskCtr
    os_core.o(.text) refers to os_cfg_app.o(.constdata) for OSCfg_IdleTaskStkSize
    os_core.o(.text) refers to os_var.o(.bss) for OSIdleTaskTCB
    os_dbg.o(.text) refers to os_dbg.o(.constdata) for OSDbg_DbgEn
    os_flag.o(.text) refers to cpu_a.o(.text) for CPU_SR_Save
    os_flag.o(.text) refers to os_core.o(.text) for OS_PendListInit
    os_flag.o(.text) refers to os_var.o(.data) for OSFlagDbgListPtr
    os_flag.o(.text) refers to bsp.o(.text) for CPU_TS_TmrRd
    os_mem.o(.text) refers to cpu_a.o(.text) for CPU_SR_Save
    os_mem.o(.text) refers to os_var.o(.data) for OSMemDbgListPtr
    os_msg.o(.text) refers to os_cfg_app.o(.constdata) for OSCfg_MsgPoolBasePtr
    os_msg.o(.text) refers to os_var.o(.bss) for OSMsgPool
    os_mutex.o(.text) refers to cpu_a.o(.text) for CPU_SR_Save
    os_mutex.o(.text) refers to os_core.o(.text) for OS_PendListInit
    os_mutex.o(.text) refers to os_prio.o(.text) for OS_PrioInsert
    os_mutex.o(.text) refers to bsp.o(.text) for CPU_TS_TmrRd
    os_mutex.o(.text) refers to os_var.o(.data) for OSMutexDbgListPtr
    os_pend_multi.o(.text) refers to os_core.o(.text) for OS_TaskBlock
    os_pend_multi.o(.text) refers to os_msg.o(.text) for OS_MsgQGet
    os_pend_multi.o(.text) refers to cpu_a.o(.text) for CPU_SR_Save
    os_pend_multi.o(.text) refers to os_var.o(.data) for OSTCBCurPtr
    os_prio.o(.text) refers to cpu_a.o(.text) for CPU_CntLeadZeros
    os_prio.o(.text) refers to os_prio.o(.data) for OSPrioTbl
    os_q.o(.text) refers to cpu_a.o(.text) for CPU_SR_Save
    os_q.o(.text) refers to os_msg.o(.text) for OS_MsgQInit
    os_q.o(.text) refers to os_core.o(.text) for OS_PendListInit
    os_q.o(.text) refers to bsp.o(.text) for CPU_TS_TmrRd
    os_q.o(.text) refers to os_var.o(.data) for OSQDbgListPtr
    os_sem.o(.text) refers to cpu_a.o(.text) for CPU_SR_Save
    os_sem.o(.text) refers to os_core.o(.text) for OS_PendListInit
    os_sem.o(.text) refers to bsp.o(.text) for CPU_TS_TmrRd
    os_sem.o(.text) refers to os_var.o(.data) for OSSemDbgListPtr
    os_task.o(.text) refers to cpu_a.o(.text) for CPU_SR_Save
    os_task.o(.text) refers to os_core.o(.text) for OS_RdyListRemove
    os_task.o(.text) refers to os_prio.o(.text) for OS_PrioInsert
    os_task.o(.text) refers to os_msg.o(.text) for OS_MsgQInit
    os_task.o(.text) refers to bsp.o(.text) for CPU_TS_TmrRd
    os_task.o(.text) refers to os_cpu_c.o(.text) for OSTaskStkInit
    os_task.o(.text) refers to os_var.o(.data) for OSIntNestingCtr
    os_task.o(.text) refers to os_cfg_app.o(.constdata) for OSCfg_StkSizeMin
    os_task.o(.text) refers to os_var.o(.bss) for OSIdleTaskTCB
    os_task.o(.text) refers to os_tick.o(.text) for OS_TickListRemove
    os_tick.o(.text) refers to cpu_a.o(.text) for CPU_SR_Save
    os_tick.o(.text) refers to bsp.o(.text) for CPU_TS_TmrRd
    os_tick.o(.text) refers to os_core.o(.text) for OS_TaskRdy
    os_tick.o(.text) refers to os_task.o(.text) for OSTaskSemPend
    os_tick.o(.text) refers to os_var.o(.data) for OSTickCtr
    os_tick.o(.text) refers to os_cfg_app.o(.constdata) for OSCfg_TickWheelSize
    os_tick.o(.text) refers to os_cfg_app.o(.bss) for OSCfg_TickWheel
    os_tick.o(.text) refers to os_var.o(.bss) for OSTickTaskTCB
    os_time.o(.text) refers to cpu_a.o(.text) for CPU_SR_Save
    os_time.o(.text) refers to os_tick.o(.text) for OS_TickListInsert
    os_time.o(.text) refers to os_core.o(.text) for OS_RdyListRemove
    os_time.o(.text) refers to os_cpu_c.o(.text) for OSTimeTickHook
    os_time.o(.text) refers to os_task.o(.text) for OSTaskSemPost
    os_time.o(.text) refers to os_var.o(.data) for OSIntNestingCtr
    os_time.o(.text) refers to os_cfg_app.o(.constdata) for OSCfg_TickRate_Hz
    os_time.o(.text) refers to os_var.o(.bss) for OSTickTaskTCB
    os_tmr.o(.text) refers to cpu_a.o(.text) for CPU_SR_Save
    os_tmr.o(.text) refers to os_core.o(.text) for OSSchedLock
    os_tmr.o(.text) refers to os_var.o(.data) for OSTmrDbgListPtr
    os_tmr.o(.text) refers to os_cfg_app.o(.constdata) for OSCfg_TmrWheelSize
    os_tmr.o(.text) refers to os_cfg_app.o(.bss) for OSCfg_TmrWheel
    os_tmr.o(.text) refers to os_task.o(.text) for OSTaskSemPend
    os_tmr.o(.text) refers to bsp.o(.text) for CPU_TS_TmrRd
    os_tmr.o(.text) refers to os_var.o(.bss) for OSTmrTaskTCB
    os_cpu_a.o(CODE) refers to os_cpu_c.o(.data) for OS_CPU_ExceptStkBase
    os_cpu_a.o(CODE) refers to os_var.o(.data) for OSTCBCurPtr
    os_cpu_a.o(CODE) refers to os_cpu_c.o(.text) for OSTaskSwHook
    os_cpu_c.o(.text) refers to bsp.o(.text) for CPU_TS_TmrRd
    os_cpu_c.o(.text) refers to cpu_a.o(.text) for CPU_SR_Save
    os_cpu_c.o(.text) refers to os_time.o(.text) for OSTimeTick
    os_cpu_c.o(.text) refers to os_core.o(.text) for OSIntExit
    os_cpu_c.o(.text) refers to os_var.o(.data) for OS_AppIdleTaskHookPtr
    os_cpu_c.o(.text) refers to os_cfg_app.o(.constdata) for OSCfg_ISRStkBasePtr
    os_cpu_c.o(.text) refers to os_cpu_c.o(.data) for OS_CPU_ExceptStkBase
    os_cpu_c.o(.text) refers to os_task.o(.text) for OS_TaskReturn
    entry.o(.ARM.Collect$$$$00000000) refers (Special) to entry10a.o(.ARM.Collect$$$$0000000D) for __rt_final_cpp
    entry.o(.ARM.Collect$$$$00000000) refers (Special) to entry11a.o(.ARM.Collect$$$$0000000F) for __rt_final_exit
    entry.o(.ARM.Collect$$$$00000000) refers (Special) to entry7b.o(.ARM.Collect$$$$00000008) for _main_clock
    entry.o(.ARM.Collect$$$$00000000) refers (Special) to entry8b.o(.ARM.Collect$$$$0000000A) for _main_cpp_init
    entry.o(.ARM.Collect$$$$00000000) refers (Special) to entry9a.o(.ARM.Collect$$$$0000000B) for _main_init
    entry.o(.ARM.Collect$$$$00000000) refers (Special) to entry5.o(.ARM.Collect$$$$00000004) for _main_scatterload
    entry.o(.ARM.Collect$$$$00000000) refers (Special) to entry2.o(.ARM.Collect$$$$00000001) for _main_stk
    uldiv.o(.text) refers to llushr.o(.text) for __aeabi_llsr
    uldiv.o(.text) refers to llshl.o(.text) for __aeabi_llsl
    entry2.o(.ARM.Collect$$$$00000001) refers to entry2.o(.ARM.Collect$$$$00002712) for __lit__00000000
    entry2.o(.ARM.Collect$$$$00002712) refers to startup_stm32f2xx.o(STACK) for __initial_sp
    entry2.o(__vectab_stack_and_reset_area) refers to startup_stm32f2xx.o(STACK) for __initial_sp
    entry2.o(__vectab_stack_and_reset_area) refers to entry.o(.ARM.Collect$$$$00000000) for __main
    entry5.o(.ARM.Collect$$$$00000004) refers to init.o(.text) for __scatterload
    entry9a.o(.ARM.Collect$$$$0000000B) refers to app.o(.text) for main
    entry9b.o(.ARM.Collect$$$$0000000C) refers to app.o(.text) for main
    init.o(.text) refers to entry5.o(.ARM.Collect$$$$00000004) for __main_after_scatterload


==============================================================================

Removing Unused input sections from the image.

    Removing os_app_hooks.o(.text), (200 bytes).
    Removing startup_stm32f2xx.o(HEAP), (512 bytes).
    Removing stm32f2xx_adc.o(.text), (1124 bytes).
    Removing stm32f2xx_dac.o(.text), (528 bytes).
    Removing stm32f2xx_dma.o(.text), (936 bytes).
    Removing stm32f2xx_exti.o(.text), (284 bytes).
    Removing stm32f2xx_fsmc.o(.text), (1544 bytes).
    Removing stm32f2xx_i2c.o(.text), (1064 bytes).
    Removing stm32f2xx_tim.o(.text), (3234 bytes).
    Removing stm32f2xx_syscfg.o(.text), (140 bytes).
    Removing stm32f2xx_iwdg.o(.text), (64 bytes).
    Removing core_cm3.o(.emb_text), (32 bytes).
    Removing lib_math.o(.text), (128 bytes).
    Removing lib_math.o(.data), (4 bytes).
    Removing os_pend_multi.o(.text), (716 bytes).

15 unused section(s) (total 10510 bytes) removed from the image.

==============================================================================

Image Symbol Table

    Local Symbols

    Symbol Name                              Value     Ov Type        Size  Object(Section)

    ../clib/microlib/division.c              0x00000000   Number         0  uldiv.o ABSOLUTE
    ../clib/microlib/init/entry.s            0x00000000   Number         0  entry.o ABSOLUTE
    ../clib/microlib/init/entry.s            0x00000000   Number         0  entry11b.o ABSOLUTE
    ../clib/microlib/init/entry.s            0x00000000   Number         0  entry8a.o ABSOLUTE
    ../clib/microlib/init/entry.s            0x00000000   Number         0  entry10b.o ABSOLUTE
    ../clib/microlib/init/entry.s            0x00000000   Number         0  entry8b.o ABSOLUTE
    ../clib/microlib/init/entry.s            0x00000000   Number         0  entry7b.o ABSOLUTE
    ../clib/microlib/init/entry.s            0x00000000   Number         0  entry9a.o ABSOLUTE
    ../clib/microlib/init/entry.s            0x00000000   Number         0  entry7a.o ABSOLUTE
    ../clib/microlib/init/entry.s            0x00000000   Number         0  entry9b.o ABSOLUTE
    ../clib/microlib/init/entry.s            0x00000000   Number         0  entry10a.o ABSOLUTE
    ../clib/microlib/init/entry.s            0x00000000   Number         0  entry5.o ABSOLUTE
    ../clib/microlib/init/entry.s            0x00000000   Number         0  entry2.o ABSOLUTE
    ../clib/microlib/init/entry.s            0x00000000   Number         0  entry11a.o ABSOLUTE
    ../clib/microlib/longlong.c              0x00000000   Number         0  llshl.o ABSOLUTE
    ../clib/microlib/longlong.c              0x00000000   Number         0  llushr.o ABSOLUTE
    ..\Libraries\CMSIS\CM3\CoreSupport\core_cm3.c 0x00000000   Number         0  core_cm3.o ABSOLUTE
    ..\Libraries\CMSIS\CM3\DeviceSupport\ST\STM32F2xx\startup\arm\startup_stm32f2xx.s 0x00000000   Number         0  startup_stm32f2xx.o ABSOLUTE
    ..\Libraries\CMSIS\CM3\DeviceSupport\ST\STM32F2xx\system_stm32f2xx.c 0x00000000   Number         0  system_stm32f2xx.o ABSOLUTE
    ..\Libraries\STM32F2xx_StdPeriph_Driver\src\misc.c 0x00000000   Number         0  misc.o ABSOLUTE
    ..\Libraries\STM32F2xx_StdPeriph_Driver\src\stm32f2xx_adc.c 0x00000000   Number         0  stm32f2xx_adc.o ABSOLUTE
    ..\Libraries\STM32F2xx_StdPeriph_Driver\src\stm32f2xx_dac.c 0x00000000   Number         0  stm32f2xx_dac.o ABSOLUTE
    ..\Libraries\STM32F2xx_StdPeriph_Driver\src\stm32f2xx_dma.c 0x00000000   Number         0  stm32f2xx_dma.o ABSOLUTE
    ..\Libraries\STM32F2xx_StdPeriph_Driver\src\stm32f2xx_exti.c 0x00000000   Number         0  stm32f2xx_exti.o ABSOLUTE
    ..\Libraries\STM32F2xx_StdPeriph_Driver\src\stm32f2xx_fsmc.c 0x00000000   Number         0  stm32f2xx_fsmc.o ABSOLUTE
    ..\Libraries\STM32F2xx_StdPeriph_Driver\src\stm32f2xx_gpio.c 0x00000000   Number         0  stm32f2xx_gpio.o ABSOLUTE
    ..\Libraries\STM32F2xx_StdPeriph_Driver\src\stm32f2xx_i2c.c 0x00000000   Number         0  stm32f2xx_i2c.o ABSOLUTE
    ..\Libraries\STM32F2xx_StdPeriph_Driver\src\stm32f2xx_iwdg.c 0x00000000   Number         0  stm32f2xx_iwdg.o ABSOLUTE
    ..\Libraries\STM32F2xx_StdPeriph_Driver\src\stm32f2xx_rcc.c 0x00000000   Number         0  stm32f2xx_rcc.o ABSOLUTE
    ..\Libraries\STM32F2xx_StdPeriph_Driver\src\stm32f2xx_syscfg.c 0x00000000   Number         0  stm32f2xx_syscfg.o ABSOLUTE
    ..\Libraries\STM32F2xx_StdPeriph_Driver\src\stm32f2xx_tim.c 0x00000000   Number         0  stm32f2xx_tim.o ABSOLUTE
    ..\Libraries\STM32F2xx_StdPeriph_Driver\src\stm32f2xx_usart.c 0x00000000   Number         0  stm32f2xx_usart.o ABSOLUTE
    ..\User\app.c                            0x00000000   Number         0  app.o ABSOLUTE
    ..\User\bsp_stm32F2xx\bsp.c              0x00000000   Number         0  bsp.o ABSOLUTE
    ..\User\bsp_stm32F2xx\bsp_int.c          0x00000000   Number         0  bsp_int.o ABSOLUTE
    ..\User\bsp_stm32F2xx\src\bsp_key.c      0x00000000   Number         0  bsp_key.o ABSOLUTE
    ..\User\bsp_stm32F2xx\src\bsp_led.c      0x00000000   Number         0  bsp_led.o ABSOLUTE
    ..\User\bsp_stm32F2xx\stm32f2xx_it.c     0x00000000   Number         0  stm32f2xx_it.o ABSOLUTE
    ..\User\os_app_hooks.c                   0x00000000   Number         0  os_app_hooks.o ABSOLUTE
    ..\\Libraries\\CMSIS\\CM3\\CoreSupport\\core_cm3.c 0x00000000   Number         0  core_cm3.o ABSOLUTE
    ..\uCOS-III\uC-CPU\ARM-Cortex-M4\RealView\cpu_a.asm 0x00000000   Number         0  cpu_a.o ABSOLUTE
    ..\uCOS-III\uC-CPU\ARM-Cortex-M4\RealView\cpu_c.c 0x00000000   Number         0  cpu_c.o ABSOLUTE
    ..\uCOS-III\uC-CPU\cpu_core.c            0x00000000   Number         0  cpu_core.o ABSOLUTE
    ..\uCOS-III\uC-LIB\Ports\ARM-Cortex-M4\RealView\lib_mem_a.asm 0x00000000   Number         0  lib_mem_a.o ABSOLUTE
    ..\uCOS-III\uC-LIB\lib_ascii.c           0x00000000   Number         0  lib_ascii.o ABSOLUTE
    ..\uCOS-III\uC-LIB\lib_math.c            0x00000000   Number         0  lib_math.o ABSOLUTE
    ..\uCOS-III\uC-LIB\lib_mem.c             0x00000000   Number         0  lib_mem.o ABSOLUTE
    ..\uCOS-III\uC-LIB\lib_str.c             0x00000000   Number         0  lib_str.o ABSOLUTE
    ..\uCOS-III\uCOS-III\Ports\ARM-Cortex-M4\Generic\RealView\os_cpu_a.asm 0x00000000   Number         0  os_cpu_a.o ABSOLUTE
    ..\uCOS-III\uCOS-III\Ports\ARM-Cortex-M4\Generic\RealView\os_cpu_c.c 0x00000000   Number         0  os_cpu_c.o ABSOLUTE
    ..\uCOS-III\uCOS-III\Source\os_cfg_app.c 0x00000000   Number         0  os_cfg_app.o ABSOLUTE
    ..\uCOS-III\uCOS-III\Source\os_core.c    0x00000000   Number         0  os_core.o ABSOLUTE
    ..\uCOS-III\uCOS-III\Source\os_dbg.c     0x00000000   Number         0  os_dbg.o ABSOLUTE
    ..\uCOS-III\uCOS-III\Source\os_flag.c    0x00000000   Number         0  os_flag.o ABSOLUTE
    ..\uCOS-III\uCOS-III\Source\os_int.c     0x00000000   Number         0  os_int.o ABSOLUTE
    ..\uCOS-III\uCOS-III\Source\os_mem.c     0x00000000   Number         0  os_mem.o ABSOLUTE
    ..\uCOS-III\uCOS-III\Source\os_msg.c     0x00000000   Number         0  os_msg.o ABSOLUTE
    ..\uCOS-III\uCOS-III\Source\os_mutex.c   0x00000000   Number         0  os_mutex.o ABSOLUTE
    ..\uCOS-III\uCOS-III\Source\os_pend_multi.c 0x00000000   Number         0  os_pend_multi.o ABSOLUTE
    ..\uCOS-III\uCOS-III\Source\os_prio.c    0x00000000   Number         0  os_prio.o ABSOLUTE
    ..\uCOS-III\uCOS-III\Source\os_q.c       0x00000000   Number         0  os_q.o ABSOLUTE
    ..\uCOS-III\uCOS-III\Source\os_sem.c     0x00000000   Number         0  os_sem.o ABSOLUTE
    ..\uCOS-III\uCOS-III\Source\os_stat.c    0x00000000   Number         0  os_stat.o ABSOLUTE
    ..\uCOS-III\uCOS-III\Source\os_task.c    0x00000000   Number         0  os_task.o ABSOLUTE
    ..\uCOS-III\uCOS-III\Source\os_tick.c    0x00000000   Number         0  os_tick.o ABSOLUTE
    ..\uCOS-III\uCOS-III\Source\os_time.c    0x00000000   Number         0  os_time.o ABSOLUTE
    ..\uCOS-III\uCOS-III\Source\os_tmr.c     0x00000000   Number         0  os_tmr.o ABSOLUTE
    ..\uCOS-III\uCOS-III\Source\os_var.c     0x00000000   Number         0  os_var.o ABSOLUTE
    dc.s                                     0x00000000   Number         0  dc.o ABSOLUTE
    handlers.s                               0x00000000   Number         0  handlers.o ABSOLUTE
    init.s                                   0x00000000   Number         0  init.o ABSOLUTE
    RESET                                    0x08000000   Section      388  startup_stm32f2xx.o(RESET)
    .ARM.Collect$$$$00000000                 0x08000184   Section        0  entry.o(.ARM.Collect$$$$00000000)
    .ARM.Collect$$$$00000001                 0x08000184   Section        4  entry2.o(.ARM.Collect$$$$00000001)
    .ARM.Collect$$$$00000004                 0x08000188   Section        4  entry5.o(.ARM.Collect$$$$00000004)
    .ARM.Collect$$$$00000008                 0x0800018c   Section        0  entry7b.o(.ARM.Collect$$$$00000008)
    .ARM.Collect$$$$0000000A                 0x0800018c   Section        0  entry8b.o(.ARM.Collect$$$$0000000A)
    .ARM.Collect$$$$0000000B                 0x0800018c   Section        8  entry9a.o(.ARM.Collect$$$$0000000B)
    .ARM.Collect$$$$0000000D                 0x08000194   Section        0  entry10a.o(.ARM.Collect$$$$0000000D)
    .ARM.Collect$$$$0000000F                 0x08000194   Section        0  entry11a.o(.ARM.Collect$$$$0000000F)
    .ARM.Collect$$$$00002712                 0x08000194   Section        4  entry2.o(.ARM.Collect$$$$00002712)
    __lit__00000000                          0x08000194   Data           4  entry2.o(.ARM.Collect$$$$00002712)
    .text                                    0x08000198   Section        0  app.o(.text)
    AppObjCreate                             0x08000199   Thumb Code    36  app.o(.text)
    AppTaskUserIF                            0x080001bd   Thumb Code    96  app.o(.text)
    AppTaskKeyScan                           0x0800021d   Thumb Code   112  app.o(.text)
    AppTaskCreate                            0x0800028d   Thumb Code   104  app.o(.text)
    AppTaskStart                             0x080002f5   Thumb Code    34  app.o(.text)
    .text                                    0x080003f8   Section        0  bsp.o(.text)
    .text                                    0x080004c0   Section        0  bsp_led.o(.text)
    .text                                    0x08000638   Section        0  stm32f2xx_it.o(.text)
    .text                                    0x08000684   Section        0  bsp_key.o(.text)
    IsKeyDown1                               0x08000685   Thumb Code    18  bsp_key.o(.text)
    IsKeyDown2                               0x08000697   Thumb Code    18  bsp_key.o(.text)
    bsp_InitKeyHard                          0x080006a9   Thumb Code    60  bsp_key.o(.text)
    bsp_InitKeyVar                           0x080006e5   Thumb Code    78  bsp_key.o(.text)
    bsp_DetectKey                            0x080007f3   Thumb Code   186  bsp_key.o(.text)
    .text                                    0x080008e0   Section        0  bsp_int.o(.text)
    BSP_IntHandlerDummy                      0x08000979   Thumb Code     2  bsp_int.o(.text)
    BSP_IntHandler                           0x08000991   Thumb Code    58  bsp_int.o(.text)
    .text                                    0x08000cfc   Section       36  startup_stm32f2xx.o(.text)
    .text                                    0x08000d20   Section        0  misc.o(.text)
    .text                                    0x08000e00   Section        0  stm32f2xx_gpio.o(.text)
    .text                                    0x0800105c   Section        0  stm32f2xx_rcc.o(.text)
    .text                                    0x080015e4   Section        0  stm32f2xx_usart.o(.text)
    .text                                    0x08001a00   Section        0  system_stm32f2xx.o(.text)
    SetSysClock                              0x08001a01   Thumb Code   192  system_stm32f2xx.o(.text)
    .text                                    0x08001be0   Section        0  cpu_core.o(.text)
    CPU_NameInit                             0x08001c0b   Thumb Code     8  cpu_core.o(.text)
    CPU_TS_Init                              0x08001c13   Thumb Code    14  cpu_core.o(.text)
    .text                                    0x08001e88   Section       52  cpu_a.o(.text)
    .text                                    0x08001ebc   Section        0  cpu_c.o(.text)
    .text                                    0x08002638   Section        0  lib_ascii.o(.text)
    .text                                    0x08002890   Section        0  lib_mem.o(.text)
    Mem_SegAlloc                             0x08002ac7   Thumb Code    80  lib_mem.o(.text)
    Mem_SegCalcTotSize                       0x08002b17   Thumb Code   164  lib_mem.o(.text)
    Mem_PoolBlkIsValidAddr                   0x0800345d   Thumb Code   102  lib_mem.o(.text)
    .text                                    0x08003754   Section        0  lib_str.o(.text)
    Str_FmtNbr_Int32                         0x08003c0d   Thumb Code   474  lib_str.o(.text)
    Str_ParseNbr_Int32                       0x08003e53   Thumb Code   446  lib_str.o(.text)
    .text                                    0x0800407c   Section      544  lib_mem_a.o(.text)
    .text                                    0x0800429c   Section        0  os_cfg_app.o(.text)
    .text                                    0x080042a0   Section        0  os_core.o(.text)
    .text                                    0x08005018   Section        0  os_dbg.o(.text)
    .text                                    0x080051c4   Section        0  os_flag.o(.text)
    .text                                    0x080058fc   Section        0  os_mem.o(.text)
    .text                                    0x08005af8   Section        0  os_msg.o(.text)
    .text                                    0x08005d20   Section        0  os_mutex.o(.text)
    .text                                    0x080061f8   Section        0  os_prio.o(.text)
    .text                                    0x08006274   Section        0  os_q.o(.text)
    .text                                    0x080067a8   Section        0  os_sem.o(.text)
    .text                                    0x08006d5c   Section        0  os_task.o(.text)
    .text                                    0x08008004   Section        0  os_tick.o(.text)
    .text                                    0x08008488   Section        0  os_time.o(.text)
    .text                                    0x08008794   Section        0  os_tmr.o(.text)
    .text                                    0x08008ed4   Section        0  os_cpu_c.o(.text)
    .text                                    0x08009134   Section        0  uldiv.o(.text)
    .text                                    0x08009196   Section        0  llshl.o(.text)
    .text                                    0x080091b4   Section        0  llushr.o(.text)
    .text                                    0x080091d4   Section       36  init.o(.text)
    CODE                                     0x080091f8   Section      152  os_cpu_a.o(CODE)
    i.__scatterload_copy                     0x08009290   Section       14  handlers.o(i.__scatterload_copy)
    i.__scatterload_null                     0x0800929e   Section        2  handlers.o(i.__scatterload_null)
    i.__scatterload_zeroinit                 0x080092a0   Section       14  handlers.o(i.__scatterload_zeroinit)
    .constdata                               0x080092ae   Section      256  cpu_core.o(.constdata)
    CPU_CntLeadZerosTbl                      0x080092ae   Data         256  cpu_core.o(.constdata)
    .constdata                               0x080093b0   Section      148  lib_str.o(.constdata)
    Str_MultOvfThTbl_Int32U                  0x080093b0   Data         148  lib_str.o(.constdata)
    .constdata                               0x08009444   Section      164  os_cfg_app.o(.constdata)
    .constdata                               0x080094e8   Section      364  os_dbg.o(.constdata)
    .data                                    0x20000000   Section        7  app.o(.data)
    .data                                    0x20000007   Section        1  bsp_key.o(.data)
    .data                                    0x20000008   Section       16  stm32f2xx_rcc.o(.data)
    APBAHBPrescTable                         0x20000008   Data          16  stm32f2xx_rcc.o(.data)
    .data                                    0x20000018   Section       20  system_stm32f2xx.o(.data)
    .data                                    0x2000002c   Section        4  cpu_core.o(.data)
    .data                                    0x20000030   Section        4  lib_mem.o(.data)
    .data                                    0x20000034   Section        4  os_prio.o(.data)
    .data                                    0x20000038   Section      156  os_var.o(.data)
    .data                                    0x200000d4   Section        4  os_cpu_c.o(.data)
    .bss                                     0x200000d8   Section    14156  app.o(.bss)
    AppTaskStartTCB                          0x200000d8   Data         196  app.o(.bss)
    AppTaskUserIFTCB                         0x2000019c   Data         196  app.o(.bss)
    AppTaskKeyScanTCB                        0x20000260   Data         196  app.o(.bss)
    AppTaskStartStk                          0x20000324   Data        4096  app.o(.bss)
    AppTaskUserIFStk                         0x20001324   Data        4096  app.o(.bss)
    AppTaskKeyScanStk                        0x20002324   Data        4096  app.o(.bss)
    .bss                                     0x20003824   Section       45  bsp_key.o(.bss)
    s_tBtn                                   0x20003824   Data          32  bsp_key.o(.bss)
    .bss                                     0x20003854   Section      324  bsp_int.o(.bss)
    BSP_IntVectTbl                           0x20003854   Data         324  bsp_int.o(.bss)
    .bss                                     0x20003998   Section       16  cpu_core.o(.bss)
    .bss                                     0x200039a8   Section     9288  lib_mem.o(.bss)
    .bss                                     0x20005df0   Section     3616  os_cfg_app.o(.bss)
    .bss                                     0x20006c10   Section      744  os_var.o(.bss)
    STACK                                    0x20006ef8   Section     1024  startup_stm32f2xx.o(STACK)

    Global Symbols

    Symbol Name                              Value     Ov Type        Size  Object(Section)

    BuildAttributes$$THM_ISAv4$P$D$K$B$S$PE$A:L22UL41UL21$X:L11$S22US41US21$IEEE1$IW$USESV6$~STKCKD$USESV7$~SHL$OSPACE$EBA8$MICROLIB$REQ8$PRES8$EABIv2 0x00000000   Number         0  anon$$obj.o ABSOLUTE
    __ARM_use_no_argv                        0x00000000   Number         0  app.o ABSOLUTE
    __cpp_initialize__aeabi_                  - Undefined Weak Reference
    __cxa_finalize                            - Undefined Weak Reference
    __decompress                              - Undefined Weak Reference
    _clock_init                               - Undefined Weak Reference
    _microlib_exit                            - Undefined Weak Reference
    __Vectors_Size                           0x00000184   Number         0  startup_stm32f2xx.o ABSOLUTE
    __Vectors                                0x08000000   Data           4  startup_stm32f2xx.o(RESET)
    __Vectors_End                            0x08000184   Data           0  startup_stm32f2xx.o(RESET)
    __main                                   0x08000185   Thumb Code     0  entry.o(.ARM.Collect$$$$00000000)
    _main_stk                                0x08000185   Thumb Code     0  entry2.o(.ARM.Collect$$$$00000001)
    _main_scatterload                        0x08000189   Thumb Code     0  entry5.o(.ARM.Collect$$$$00000004)
    __main_after_scatterload                 0x0800018d   Thumb Code     0  entry5.o(.ARM.Collect$$$$00000004)
    _main_clock                              0x0800018d   Thumb Code     0  entry7b.o(.ARM.Collect$$$$00000008)
    _main_cpp_init                           0x0800018d   Thumb Code     0  entry8b.o(.ARM.Collect$$$$0000000A)
    _main_init                               0x0800018d   Thumb Code     0  entry9a.o(.ARM.Collect$$$$0000000B)
    __rt_final_cpp                           0x08000195   Thumb Code     0  entry10a.o(.ARM.Collect$$$$0000000D)
    __rt_final_exit                          0x08000195   Thumb Code     0  entry11a.o(.ARM.Collect$$$$0000000F)
    main                                     0x08000317   Thumb Code    78  app.o(.text)
    NVIC_Configuration                       0x080003f9   Thumb Code    12  bsp.o(.text)
    bsp_Init                                 0x08000405   Thumb Code    16  bsp.o(.text)
    bsp_RunPer10ms                           0x08000415   Thumb Code     8  bsp.o(.text)
    bsp_RunPer1ms                            0x0800041d   Thumb Code     2  bsp.o(.text)
    bsp_Idle                                 0x0800041f   Thumb Code     2  bsp.o(.text)
    BSP_CPU_ClkFreq                          0x08000421   Thumb Code    14  bsp.o(.text)
    BSP_Tick_Init                            0x0800042f   Thumb Code    24  bsp.o(.text)
    CPU_TS_TmrInit                           0x08000447   Thumb Code    44  bsp.o(.text)
    CPU_TS_TmrRd                             0x08000473   Thumb Code     6  bsp.o(.text)
    CPU_TS32_to_uSec                         0x08000479   Thumb Code    54  bsp.o(.text)
    bsp_LedOff                               0x080004c1   Thumb Code    50  bsp_led.o(.text)
    bsp_InitLed                              0x080004f3   Thumb Code   106  bsp_led.o(.text)
    bsp_LedOn                                0x0800055d   Thumb Code    50  bsp_led.o(.text)
    bsp_LedToggle                            0x0800058f   Thumb Code    72  bsp_led.o(.text)
    bsp_IsLedOn                              0x080005d7   Thumb Code    94  bsp_led.o(.text)
    NMI_Handler                              0x08000639   Thumb Code     2  stm32f2xx_it.o(.text)
    HardFault_Handler                        0x0800063b   Thumb Code    16  stm32f2xx_it.o(.text)
    MemManage_Handler                        0x0800064b   Thumb Code     4  stm32f2xx_it.o(.text)
    BusFault_Handler                         0x0800064f   Thumb Code     4  stm32f2xx_it.o(.text)
    UsageFault_Handler                       0x08000653   Thumb Code     4  stm32f2xx_it.o(.text)
    SVC_Handler                              0x08000657   Thumb Code     2  stm32f2xx_it.o(.text)
    DebugMon_Handler                         0x08000659   Thumb Code     2  stm32f2xx_it.o(.text)
    PendSV_Handler                           0x0800065b   Thumb Code     2  stm32f2xx_it.o(.text)
    USART3_IRQHandler                        0x0800065d   Thumb Code    32  stm32f2xx_it.o(.text)
    bsp_InitKey                              0x08000733   Thumb Code    12  bsp_key.o(.text)
    bsp_PutKey                               0x0800073f   Thumb Code    28  bsp_key.o(.text)
    bsp_GetKey                               0x0800075b   Thumb Code    54  bsp_key.o(.text)
    bsp_GetKey2                              0x08000791   Thumb Code    46  bsp_key.o(.text)
    bsp_GetKeyState                          0x080007bf   Thumb Code    12  bsp_key.o(.text)
    bsp_SetKeyParam                          0x080007cb   Thumb Code    30  bsp_key.o(.text)
    bsp_ClearKey                             0x080007e9   Thumb Code    10  bsp_key.o(.text)
    bsp_KeyScan                              0x080008ad   Thumb Code    22  bsp_key.o(.text)
    BSP_IntClr                               0x080008e1   Thumb Code     2  bsp_int.o(.text)
    BSP_IntDis                               0x080008e3   Thumb Code    20  bsp_int.o(.text)
    BSP_IntDisAll                            0x080008f7   Thumb Code     8  bsp_int.o(.text)
    BSP_IntEn                                0x080008ff   Thumb Code    20  bsp_int.o(.text)
    BSP_IntVectSet                           0x08000913   Thumb Code    48  bsp_int.o(.text)
    BSP_IntPrioSet                           0x08000943   Thumb Code    54  bsp_int.o(.text)
    BSP_IntInit                              0x0800097b   Thumb Code    22  bsp_int.o(.text)
    BSP_IntHandlerWWDG                       0x080009cb   Thumb Code    10  bsp_int.o(.text)
    BSP_IntHandlerPVD                        0x080009d5   Thumb Code    10  bsp_int.o(.text)
    BSP_IntHandlerTAMPER                     0x080009df   Thumb Code    10  bsp_int.o(.text)
    BSP_IntHandlerRTC                        0x080009e9   Thumb Code    10  bsp_int.o(.text)
    BSP_IntHandlerFLASH                      0x080009f3   Thumb Code    10  bsp_int.o(.text)
    BSP_IntHandlerRCC                        0x080009fd   Thumb Code    10  bsp_int.o(.text)
    BSP_IntHandlerEXTI0                      0x08000a07   Thumb Code    10  bsp_int.o(.text)
    BSP_IntHandlerEXTI1                      0x08000a11   Thumb Code    10  bsp_int.o(.text)
    BSP_IntHandlerEXTI2                      0x08000a1b   Thumb Code    10  bsp_int.o(.text)
    BSP_IntHandlerEXTI3                      0x08000a25   Thumb Code    10  bsp_int.o(.text)
    BSP_IntHandlerEXTI4                      0x08000a2f   Thumb Code    10  bsp_int.o(.text)
    BSP_IntHandlerDMA1_CH1                   0x08000a39   Thumb Code    10  bsp_int.o(.text)
    BSP_IntHandlerDMA1_CH2                   0x08000a43   Thumb Code    10  bsp_int.o(.text)
    BSP_IntHandlerDMA1_CH3                   0x08000a4d   Thumb Code    10  bsp_int.o(.text)
    BSP_IntHandlerDMA1_CH4                   0x08000a57   Thumb Code    10  bsp_int.o(.text)
    BSP_IntHandlerDMA1_CH5                   0x08000a61   Thumb Code    10  bsp_int.o(.text)
    BSP_IntHandlerDMA1_CH6                   0x08000a6b   Thumb Code    10  bsp_int.o(.text)
    BSP_IntHandlerDMA1_CH7                   0x08000a75   Thumb Code    10  bsp_int.o(.text)
    BSP_IntHandlerADC1_2                     0x08000a7f   Thumb Code    10  bsp_int.o(.text)
    BSP_IntHandlerCAN1_TX                    0x08000a89   Thumb Code    10  bsp_int.o(.text)
    BSP_IntHandlerCAN1_RX0                   0x08000a93   Thumb Code    10  bsp_int.o(.text)
    BSP_IntHandlerCAN1_RX1                   0x08000a9d   Thumb Code    10  bsp_int.o(.text)
    BSP_IntHandlerCAN1_SCE                   0x08000aa7   Thumb Code    10  bsp_int.o(.text)
    BSP_IntHandlerEXTI9_5                    0x08000ab1   Thumb Code    10  bsp_int.o(.text)
    BSP_IntHandlerTIM1_BRK                   0x08000abb   Thumb Code    10  bsp_int.o(.text)
    BSP_IntHandlerTIM1_UP                    0x08000ac5   Thumb Code    10  bsp_int.o(.text)
    BSP_IntHandlerTIM1_TRG_COM               0x08000acf   Thumb Code    10  bsp_int.o(.text)
    BSP_IntHandlerTIM1_CC                    0x08000ad9   Thumb Code    10  bsp_int.o(.text)
    BSP_IntHandlerTIM2                       0x08000ae3   Thumb Code    10  bsp_int.o(.text)
    BSP_IntHandlerTIM3                       0x08000aed   Thumb Code    10  bsp_int.o(.text)
    BSP_IntHandlerTIM4                       0x08000af7   Thumb Code    10  bsp_int.o(.text)
    BSP_IntHandlerI2C1_EV                    0x08000b01   Thumb Code    10  bsp_int.o(.text)
    BSP_IntHandlerI2C1_ER                    0x08000b0b   Thumb Code    10  bsp_int.o(.text)
    BSP_IntHandlerI2C2_EV                    0x08000b15   Thumb Code    10  bsp_int.o(.text)
    BSP_IntHandlerI2C2_ER                    0x08000b1f   Thumb Code    10  bsp_int.o(.text)
    BSP_IntHandlerSPI1                       0x08000b29   Thumb Code    10  bsp_int.o(.text)
    BSP_IntHandlerSPI2                       0x08000b33   Thumb Code    10  bsp_int.o(.text)
    BSP_IntHandlerUSART1                     0x08000b3d   Thumb Code    10  bsp_int.o(.text)
    BSP_IntHandlerUSART2                     0x08000b47   Thumb Code    10  bsp_int.o(.text)
    BSP_IntHandlerUSART3                     0x08000b51   Thumb Code    10  bsp_int.o(.text)
    BSP_IntHandlerEXTI15_10                  0x08000b5b   Thumb Code    10  bsp_int.o(.text)
    BSP_IntHandlerRTCAlarm                   0x08000b65   Thumb Code    10  bsp_int.o(.text)
    BSP_IntHandlerUSBWakeUp                  0x08000b6f   Thumb Code    10  bsp_int.o(.text)
    BSP_IntHandlerTIM8_BRK_TIM12             0x08000b79   Thumb Code    10  bsp_int.o(.text)
    BSP_IntHandlerTIM8_UP_TIM13              0x08000b83   Thumb Code    10  bsp_int.o(.text)
    BSP_IntHandlerTIM8_TRG_COM_TIM14         0x08000b8d   Thumb Code    10  bsp_int.o(.text)
    BSP_IntHandlerTIM8_CC                    0x08000b97   Thumb Code    10  bsp_int.o(.text)
    BSP_IntHandlerDMA1_STREAM7               0x08000ba1   Thumb Code    10  bsp_int.o(.text)
    BSP_IntHandlerFSMC                       0x08000bab   Thumb Code    10  bsp_int.o(.text)
    BSP_IntHandlerSDIO                       0x08000bb5   Thumb Code    10  bsp_int.o(.text)
    BSP_IntHandlerTIM5                       0x08000bbf   Thumb Code    10  bsp_int.o(.text)
    BSP_IntHandlerSPI3                       0x08000bc9   Thumb Code    10  bsp_int.o(.text)
    BSP_IntHandlerUSART4                     0x08000bd3   Thumb Code    10  bsp_int.o(.text)
    BSP_IntHandlerUSART5                     0x08000bdd   Thumb Code    10  bsp_int.o(.text)
    BSP_IntHandlerTIM6                       0x08000be7   Thumb Code    10  bsp_int.o(.text)
    BSP_IntHandlerTIM7                       0x08000bf1   Thumb Code    10  bsp_int.o(.text)
    BSP_IntHandlerDMA2_CH1                   0x08000bfb   Thumb Code    10  bsp_int.o(.text)
    BSP_IntHandlerDMA2_CH2                   0x08000c05   Thumb Code    10  bsp_int.o(.text)
    BSP_IntHandlerDMA2_CH3                   0x08000c0f   Thumb Code    10  bsp_int.o(.text)
    BSP_IntHandlerDMA2_CH4                   0x08000c19   Thumb Code    10  bsp_int.o(.text)
    BSP_IntHandlerDMA2_CH5                   0x08000c23   Thumb Code    10  bsp_int.o(.text)
    BSP_IntHandlerETH                        0x08000c2d   Thumb Code    10  bsp_int.o(.text)
    BSP_IntHandlerETHWakeup                  0x08000c37   Thumb Code    10  bsp_int.o(.text)
    BSP_IntHandlerCAN2_TX                    0x08000c41   Thumb Code    10  bsp_int.o(.text)
    BSP_IntHandlerCAN2_RX0                   0x08000c4b   Thumb Code    10  bsp_int.o(.text)
    BSP_IntHandlerCAN2_RX1                   0x08000c55   Thumb Code    10  bsp_int.o(.text)
    BSP_IntHandlerCAN2_SCE                   0x08000c5f   Thumb Code    10  bsp_int.o(.text)
    BSP_IntHandlerOTG                        0x08000c69   Thumb Code    10  bsp_int.o(.text)
    BSP_IntHandlerDMA2_CH6                   0x08000c73   Thumb Code    10  bsp_int.o(.text)
    BSP_IntHandlerDMA2_CH7                   0x08000c7d   Thumb Code    10  bsp_int.o(.text)
    BSP_IntHandlerDMA2_CH8                   0x08000c87   Thumb Code    10  bsp_int.o(.text)
    BSP_IntHandlerUSART6                     0x08000c91   Thumb Code    10  bsp_int.o(.text)
    BSP_IntHandlerI2C3_EV                    0x08000c9b   Thumb Code    10  bsp_int.o(.text)
    BSP_IntHandlerI2C3_ER                    0x08000ca5   Thumb Code    10  bsp_int.o(.text)
    BSP_IntHandlerOTG_HS_EP1_OUT             0x08000caf   Thumb Code    10  bsp_int.o(.text)
    BSP_IntHandlerOTG_HS_EP1_IN              0x08000cb9   Thumb Code    10  bsp_int.o(.text)
    BSP_IntHandlerOTG_HS_WKUP                0x08000cc3   Thumb Code    10  bsp_int.o(.text)
    BSP_IntHandlerOTG_HS                     0x08000ccd   Thumb Code    10  bsp_int.o(.text)
    BSP_IntHandlerDCMI                       0x08000cd7   Thumb Code    10  bsp_int.o(.text)
    BSP_IntHandlerCRYP                       0x08000ce1   Thumb Code    10  bsp_int.o(.text)
    BSP_IntHandlerHASH_RNG                   0x08000ceb   Thumb Code    10  bsp_int.o(.text)
    Reset_Handler                            0x08000cfd   Thumb Code     8  startup_stm32f2xx.o(.text)
    ADC_IRQHandler                           0x08000d17   Thumb Code     0  startup_stm32f2xx.o(.text)
    CAN1_RX0_IRQHandler                      0x08000d17   Thumb Code     0  startup_stm32f2xx.o(.text)
    CAN1_RX1_IRQHandler                      0x08000d17   Thumb Code     0  startup_stm32f2xx.o(.text)
    CAN1_SCE_IRQHandler                      0x08000d17   Thumb Code     0  startup_stm32f2xx.o(.text)
    CAN1_TX_IRQHandler                       0x08000d17   Thumb Code     0  startup_stm32f2xx.o(.text)
    CAN2_RX0_IRQHandler                      0x08000d17   Thumb Code     0  startup_stm32f2xx.o(.text)
    CAN2_RX1_IRQHandler                      0x08000d17   Thumb Code     0  startup_stm32f2xx.o(.text)
    CAN2_SCE_IRQHandler                      0x08000d17   Thumb Code     0  startup_stm32f2xx.o(.text)
    CAN2_TX_IRQHandler                       0x08000d17   Thumb Code     0  startup_stm32f2xx.o(.text)
    CRYP_IRQHandler                          0x08000d17   Thumb Code     0  startup_stm32f2xx.o(.text)
    DCMI_IRQHandler                          0x08000d17   Thumb Code     0  startup_stm32f2xx.o(.text)
    DMA1_Stream0_IRQHandler                  0x08000d17   Thumb Code     0  startup_stm32f2xx.o(.text)
    DMA1_Stream1_IRQHandler                  0x08000d17   Thumb Code     0  startup_stm32f2xx.o(.text)
    DMA1_Stream2_IRQHandler                  0x08000d17   Thumb Code     0  startup_stm32f2xx.o(.text)
    DMA1_Stream3_IRQHandler                  0x08000d17   Thumb Code     0  startup_stm32f2xx.o(.text)
    DMA1_Stream4_IRQHandler                  0x08000d17   Thumb Code     0  startup_stm32f2xx.o(.text)
    DMA1_Stream5_IRQHandler                  0x08000d17   Thumb Code     0  startup_stm32f2xx.o(.text)
    DMA1_Stream6_IRQHandler                  0x08000d17   Thumb Code     0  startup_stm32f2xx.o(.text)
    DMA1_Stream7_IRQHandler                  0x08000d17   Thumb Code     0  startup_stm32f2xx.o(.text)
    DMA2_Stream0_IRQHandler                  0x08000d17   Thumb Code     0  startup_stm32f2xx.o(.text)
    DMA2_Stream1_IRQHandler                  0x08000d17   Thumb Code     0  startup_stm32f2xx.o(.text)
    DMA2_Stream2_IRQHandler                  0x08000d17   Thumb Code     0  startup_stm32f2xx.o(.text)
    DMA2_Stream3_IRQHandler                  0x08000d17   Thumb Code     0  startup_stm32f2xx.o(.text)
    DMA2_Stream4_IRQHandler                  0x08000d17   Thumb Code     0  startup_stm32f2xx.o(.text)
    DMA2_Stream5_IRQHandler                  0x08000d17   Thumb Code     0  startup_stm32f2xx.o(.text)
    DMA2_Stream6_IRQHandler                  0x08000d17   Thumb Code     0  startup_stm32f2xx.o(.text)
    DMA2_Stream7_IRQHandler                  0x08000d17   Thumb Code     0  startup_stm32f2xx.o(.text)
    ETH_IRQHandler                           0x08000d17   Thumb Code     0  startup_stm32f2xx.o(.text)
    ETH_WKUP_IRQHandler                      0x08000d17   Thumb Code     0  startup_stm32f2xx.o(.text)
    EXTI0_IRQHandler                         0x08000d17   Thumb Code     0  startup_stm32f2xx.o(.text)
    EXTI15_10_IRQHandler                     0x08000d17   Thumb Code     0  startup_stm32f2xx.o(.text)
    EXTI1_IRQHandler                         0x08000d17   Thumb Code     0  startup_stm32f2xx.o(.text)
    EXTI2_IRQHandler                         0x08000d17   Thumb Code     0  startup_stm32f2xx.o(.text)
    EXTI3_IRQHandler                         0x08000d17   Thumb Code     0  startup_stm32f2xx.o(.text)
    EXTI4_IRQHandler                         0x08000d17   Thumb Code     0  startup_stm32f2xx.o(.text)
    EXTI9_5_IRQHandler                       0x08000d17   Thumb Code     0  startup_stm32f2xx.o(.text)
    FLASH_IRQHandler                         0x08000d17   Thumb Code     0  startup_stm32f2xx.o(.text)
    FSMC_IRQHandler                          0x08000d17   Thumb Code     0  startup_stm32f2xx.o(.text)
    HASH_RNG_IRQHandler                      0x08000d17   Thumb Code     0  startup_stm32f2xx.o(.text)
    I2C1_ER_IRQHandler                       0x08000d17   Thumb Code     0  startup_stm32f2xx.o(.text)
    I2C1_EV_IRQHandler                       0x08000d17   Thumb Code     0  startup_stm32f2xx.o(.text)
    I2C2_ER_IRQHandler                       0x08000d17   Thumb Code     0  startup_stm32f2xx.o(.text)
    I2C2_EV_IRQHandler                       0x08000d17   Thumb Code     0  startup_stm32f2xx.o(.text)
    I2C3_ER_IRQHandler                       0x08000d17   Thumb Code     0  startup_stm32f2xx.o(.text)
    I2C3_EV_IRQHandler                       0x08000d17   Thumb Code     0  startup_stm32f2xx.o(.text)
    OTG_FS_IRQHandler                        0x08000d17   Thumb Code     0  startup_stm32f2xx.o(.text)
    OTG_FS_WKUP_IRQHandler                   0x08000d17   Thumb Code     0  startup_stm32f2xx.o(.text)
    OTG_HS_EP1_IN_IRQHandler                 0x08000d17   Thumb Code     0  startup_stm32f2xx.o(.text)
    OTG_HS_EP1_OUT_IRQHandler                0x08000d17   Thumb Code     0  startup_stm32f2xx.o(.text)
    OTG_HS_IRQHandler                        0x08000d17   Thumb Code     0  startup_stm32f2xx.o(.text)
    OTG_HS_WKUP_IRQHandler                   0x08000d17   Thumb Code     0  startup_stm32f2xx.o(.text)
    PVD_IRQHandler                           0x08000d17   Thumb Code     0  startup_stm32f2xx.o(.text)
    RCC_IRQHandler                           0x08000d17   Thumb Code     0  startup_stm32f2xx.o(.text)
    RTC_Alarm_IRQHandler                     0x08000d17   Thumb Code     0  startup_stm32f2xx.o(.text)
    RTC_WKUP_IRQHandler                      0x08000d17   Thumb Code     0  startup_stm32f2xx.o(.text)
    SDIO_IRQHandler                          0x08000d17   Thumb Code     0  startup_stm32f2xx.o(.text)
    SPI1_IRQHandler                          0x08000d17   Thumb Code     0  startup_stm32f2xx.o(.text)
    SPI2_IRQHandler                          0x08000d17   Thumb Code     0  startup_stm32f2xx.o(.text)
    SPI3_IRQHandler                          0x08000d17   Thumb Code     0  startup_stm32f2xx.o(.text)
    TAMP_STAMP_IRQHandler                    0x08000d17   Thumb Code     0  startup_stm32f2xx.o(.text)
    TIM1_BRK_TIM9_IRQHandler                 0x08000d17   Thumb Code     0  startup_stm32f2xx.o(.text)
    TIM1_CC_IRQHandler                       0x08000d17   Thumb Code     0  startup_stm32f2xx.o(.text)
    TIM1_TRG_COM_TIM11_IRQHandler            0x08000d17   Thumb Code     0  startup_stm32f2xx.o(.text)
    TIM1_UP_TIM10_IRQHandler                 0x08000d17   Thumb Code     0  startup_stm32f2xx.o(.text)
    TIM2_IRQHandler                          0x08000d17   Thumb Code     0  startup_stm32f2xx.o(.text)
    TIM3_IRQHandler                          0x08000d17   Thumb Code     0  startup_stm32f2xx.o(.text)
    TIM4_IRQHandler                          0x08000d17   Thumb Code     0  startup_stm32f2xx.o(.text)
    TIM5_IRQHandler                          0x08000d17   Thumb Code     0  startup_stm32f2xx.o(.text)
    TIM6_DAC_IRQHandler                      0x08000d17   Thumb Code     0  startup_stm32f2xx.o(.text)
    TIM7_IRQHandler                          0x08000d17   Thumb Code     0  startup_stm32f2xx.o(.text)
    TIM8_BRK_TIM12_IRQHandler                0x08000d17   Thumb Code     0  startup_stm32f2xx.o(.text)
    TIM8_CC_IRQHandler                       0x08000d17   Thumb Code     0  startup_stm32f2xx.o(.text)
    TIM8_TRG_COM_TIM14_IRQHandler            0x08000d17   Thumb Code     0  startup_stm32f2xx.o(.text)
    TIM8_UP_TIM13_IRQHandler                 0x08000d17   Thumb Code     0  startup_stm32f2xx.o(.text)
    UART4_IRQHandler                         0x08000d17   Thumb Code     0  startup_stm32f2xx.o(.text)
    UART5_IRQHandler                         0x08000d17   Thumb Code     0  startup_stm32f2xx.o(.text)
    USART1_IRQHandler                        0x08000d17   Thumb Code     0  startup_stm32f2xx.o(.text)
    USART2_IRQHandler                        0x08000d17   Thumb Code     0  startup_stm32f2xx.o(.text)
    USART6_IRQHandler                        0x08000d17   Thumb Code     0  startup_stm32f2xx.o(.text)
    WWDG_IRQHandler                          0x08000d17   Thumb Code     0  startup_stm32f2xx.o(.text)
    NVIC_PriorityGroupConfig                 0x08000d21   Thumb Code    10  misc.o(.text)
    NVIC_Init                                0x08000d2b   Thumb Code   106  misc.o(.text)
    NVIC_SetVectorTable                      0x08000d95   Thumb Code    14  misc.o(.text)
    NVIC_SystemLPConfig                      0x08000da3   Thumb Code    34  misc.o(.text)
    SysTick_CLKSourceConfig                  0x08000dc5   Thumb Code    40  misc.o(.text)
    GPIO_DeInit                              0x08000e01   Thumb Code   220  stm32f2xx_gpio.o(.text)
    GPIO_Init                                0x08000edd   Thumb Code   144  stm32f2xx_gpio.o(.text)
    GPIO_StructInit                          0x08000f6d   Thumb Code    18  stm32f2xx_gpio.o(.text)
    GPIO_PinLockConfig                       0x08000f7f   Thumb Code    34  stm32f2xx_gpio.o(.text)
    GPIO_ReadInputDataBit                    0x08000fa1   Thumb Code    18  stm32f2xx_gpio.o(.text)
    GPIO_ReadInputData                       0x08000fb3   Thumb Code     8  stm32f2xx_gpio.o(.text)
    GPIO_ReadOutputDataBit                   0x08000fbb   Thumb Code    18  stm32f2xx_gpio.o(.text)
    GPIO_ReadOutputData                      0x08000fcd   Thumb Code     8  stm32f2xx_gpio.o(.text)
    GPIO_SetBits                             0x08000fd5   Thumb Code     4  stm32f2xx_gpio.o(.text)
    GPIO_ResetBits                           0x08000fd9   Thumb Code     4  stm32f2xx_gpio.o(.text)
    GPIO_WriteBit                            0x08000fdd   Thumb Code    10  stm32f2xx_gpio.o(.text)
    GPIO_Write                               0x08000fe7   Thumb Code     4  stm32f2xx_gpio.o(.text)
    GPIO_ToggleBits                          0x08000feb   Thumb Code     8  stm32f2xx_gpio.o(.text)
    GPIO_PinAFConfig                         0x08000ff3   Thumb Code    70  stm32f2xx_gpio.o(.text)
    RCC_DeInit                               0x0800105d   Thumb Code    60  stm32f2xx_rcc.o(.text)
    RCC_HSEConfig                            0x08001099   Thumb Code    14  stm32f2xx_rcc.o(.text)
    RCC_GetFlagStatus                        0x080010a7   Thumb Code    60  stm32f2xx_rcc.o(.text)
    RCC_WaitForHSEStartUp                    0x080010e3   Thumb Code    56  stm32f2xx_rcc.o(.text)
    RCC_AdjustHSICalibrationValue            0x0800111b   Thumb Code    20  stm32f2xx_rcc.o(.text)
    RCC_HSICmd                               0x0800112f   Thumb Code     6  stm32f2xx_rcc.o(.text)
    RCC_LSEConfig                            0x08001135   Thumb Code    46  stm32f2xx_rcc.o(.text)
    RCC_LSICmd                               0x08001163   Thumb Code     6  stm32f2xx_rcc.o(.text)
    RCC_PLLConfig                            0x08001169   Thumb Code    32  stm32f2xx_rcc.o(.text)
    RCC_PLLCmd                               0x08001189   Thumb Code     6  stm32f2xx_rcc.o(.text)
    RCC_PLLI2SConfig                         0x0800118f   Thumb Code    14  stm32f2xx_rcc.o(.text)
    RCC_PLLI2SCmd                            0x0800119d   Thumb Code     6  stm32f2xx_rcc.o(.text)
    RCC_ClockSecuritySystemCmd               0x080011a3   Thumb Code     6  stm32f2xx_rcc.o(.text)
    RCC_MCO1Config                           0x080011a9   Thumb Code    28  stm32f2xx_rcc.o(.text)
    RCC_MCO2Config                           0x080011c5   Thumb Code    28  stm32f2xx_rcc.o(.text)
    RCC_SYSCLKConfig                         0x080011e1   Thumb Code    20  stm32f2xx_rcc.o(.text)
    RCC_GetSYSCLKSource                      0x080011f5   Thumb Code    12  stm32f2xx_rcc.o(.text)
    RCC_HCLKConfig                           0x08001201   Thumb Code    20  stm32f2xx_rcc.o(.text)
    RCC_PCLK1Config                          0x08001215   Thumb Code    20  stm32f2xx_rcc.o(.text)
    RCC_PCLK2Config                          0x08001229   Thumb Code    22  stm32f2xx_rcc.o(.text)
    RCC_GetClocksFreq                        0x0800123f   Thumb Code   222  stm32f2xx_rcc.o(.text)
    RCC_RTCCLKConfig                         0x0800131d   Thumb Code    54  stm32f2xx_rcc.o(.text)
    RCC_RTCCLKCmd                            0x08001353   Thumb Code     8  stm32f2xx_rcc.o(.text)
    RCC_BackupResetCmd                       0x0800135b   Thumb Code     8  stm32f2xx_rcc.o(.text)
    RCC_I2SCLKConfig                         0x08001363   Thumb Code     6  stm32f2xx_rcc.o(.text)
    RCC_AHB1PeriphClockCmd                   0x08001369   Thumb Code    34  stm32f2xx_rcc.o(.text)
    RCC_AHB2PeriphClockCmd                   0x0800138b   Thumb Code    34  stm32f2xx_rcc.o(.text)
    RCC_AHB3PeriphClockCmd                   0x080013ad   Thumb Code    34  stm32f2xx_rcc.o(.text)
    RCC_APB1PeriphClockCmd                   0x080013cf   Thumb Code    34  stm32f2xx_rcc.o(.text)
    RCC_APB2PeriphClockCmd                   0x080013f1   Thumb Code    34  stm32f2xx_rcc.o(.text)
    RCC_AHB1PeriphResetCmd                   0x08001413   Thumb Code    34  stm32f2xx_rcc.o(.text)
    RCC_AHB2PeriphResetCmd                   0x08001435   Thumb Code    72  stm32f2xx_rcc.o(.text)
    RCC_AHB3PeriphResetCmd                   0x0800147d   Thumb Code    34  stm32f2xx_rcc.o(.text)
    RCC_APB1PeriphResetCmd                   0x0800149f   Thumb Code    34  stm32f2xx_rcc.o(.text)
    RCC_APB2PeriphResetCmd                   0x080014c1   Thumb Code    34  stm32f2xx_rcc.o(.text)
    RCC_AHB1PeriphClockLPModeCmd             0x080014e3   Thumb Code    34  stm32f2xx_rcc.o(.text)
    RCC_AHB2PeriphClockLPModeCmd             0x08001505   Thumb Code    34  stm32f2xx_rcc.o(.text)
    RCC_AHB3PeriphClockLPModeCmd             0x08001527   Thumb Code    34  stm32f2xx_rcc.o(.text)
    RCC_APB1PeriphClockLPModeCmd             0x08001549   Thumb Code    34  stm32f2xx_rcc.o(.text)
    RCC_APB2PeriphClockLPModeCmd             0x0800156b   Thumb Code    34  stm32f2xx_rcc.o(.text)
    RCC_ITConfig                             0x0800158d   Thumb Code    34  stm32f2xx_rcc.o(.text)
    RCC_ClearFlag                            0x080015af   Thumb Code    18  stm32f2xx_rcc.o(.text)
    RCC_GetITStatus                          0x080015c1   Thumb Code    22  stm32f2xx_rcc.o(.text)
    RCC_ClearITPendingBit                    0x080015d7   Thumb Code     8  stm32f2xx_rcc.o(.text)
    USART_DeInit                             0x080015e5   Thumb Code   156  stm32f2xx_usart.o(.text)
    USART_Init                               0x08001681   Thumb Code   204  stm32f2xx_usart.o(.text)
    USART_StructInit                         0x0800174d   Thumb Code    24  stm32f2xx_usart.o(.text)
    USART_ClockInit                          0x08001765   Thumb Code    32  stm32f2xx_usart.o(.text)
    USART_ClockStructInit                    0x08001785   Thumb Code    12  stm32f2xx_usart.o(.text)
    USART_Cmd                                0x08001791   Thumb Code    24  stm32f2xx_usart.o(.text)
    USART_SetPrescaler                       0x080017a9   Thumb Code    16  stm32f2xx_usart.o(.text)
    USART_OverSampling8Cmd                   0x080017b9   Thumb Code    22  stm32f2xx_usart.o(.text)
    USART_OneBitMethodCmd                    0x080017cf   Thumb Code    24  stm32f2xx_usart.o(.text)
    USART_SendData                           0x080017e7   Thumb Code     8  stm32f2xx_usart.o(.text)
    USART_ReceiveData                        0x080017ef   Thumb Code    10  stm32f2xx_usart.o(.text)
    USART_SetAddress                         0x080017f9   Thumb Code    18  stm32f2xx_usart.o(.text)
    USART_ReceiverWakeUpCmd                  0x0800180b   Thumb Code    24  stm32f2xx_usart.o(.text)
    USART_WakeUpConfig                       0x08001823   Thumb Code    18  stm32f2xx_usart.o(.text)
    USART_LINBreakDetectLengthConfig         0x08001835   Thumb Code    18  stm32f2xx_usart.o(.text)
    USART_LINCmd                             0x08001847   Thumb Code    24  stm32f2xx_usart.o(.text)
    USART_SendBreak                          0x0800185f   Thumb Code    10  stm32f2xx_usart.o(.text)
    USART_HalfDuplexCmd                      0x08001869   Thumb Code    24  stm32f2xx_usart.o(.text)
    USART_SetGuardTime                       0x08001881   Thumb Code    16  stm32f2xx_usart.o(.text)
    USART_SmartCardCmd                       0x08001891   Thumb Code    24  stm32f2xx_usart.o(.text)
    USART_SmartCardNACKCmd                   0x080018a9   Thumb Code    24  stm32f2xx_usart.o(.text)
    USART_IrDAConfig                         0x080018c1   Thumb Code    18  stm32f2xx_usart.o(.text)
    USART_IrDACmd                            0x080018d3   Thumb Code    24  stm32f2xx_usart.o(.text)
    USART_DMACmd                             0x080018eb   Thumb Code    18  stm32f2xx_usart.o(.text)
    USART_ITConfig                           0x080018fd   Thumb Code    74  stm32f2xx_usart.o(.text)
    USART_GetFlagStatus                      0x08001947   Thumb Code    26  stm32f2xx_usart.o(.text)
    USART_ClearFlag                          0x08001961   Thumb Code    18  stm32f2xx_usart.o(.text)
    USART_GetITStatus                        0x08001973   Thumb Code   110  stm32f2xx_usart.o(.text)
    USART_ClearITPendingBit                  0x080019e1   Thumb Code    30  stm32f2xx_usart.o(.text)
    SystemInit                               0x08001ac1   Thumb Code    74  system_stm32f2xx.o(.text)
    SystemCoreClockUpdate                    0x08001b0b   Thumb Code   174  system_stm32f2xx.o(.text)
    CPU_NameClr                              0x08001be1   Thumb Code    42  cpu_core.o(.text)
    CPU_Init                                 0x08001c21   Thumb Code    12  cpu_core.o(.text)
    CPU_SW_Exception                         0x08001c2d   Thumb Code     4  cpu_core.o(.text)
    CPU_NameGet                              0x08001c31   Thumb Code    70  cpu_core.o(.text)
    CPU_NameSet                              0x08001c77   Thumb Code    96  cpu_core.o(.text)
    CPU_TS_Get32                             0x08001cd7   Thumb Code    12  cpu_core.o(.text)
    CPU_TS_Update                            0x08001ce3   Thumb Code     2  cpu_core.o(.text)
    CPU_TS_TmrFreqGet                        0x08001ce5   Thumb Code    30  cpu_core.o(.text)
    CPU_TS_TmrFreqSet                        0x08001d03   Thumb Code     6  cpu_core.o(.text)
    CPU_CntLeadZeros08                       0x08001d09   Thumb Code    18  cpu_core.o(.text)
    CPU_CntLeadZeros16                       0x08001d1b   Thumb Code    18  cpu_core.o(.text)
    CPU_CntLeadZeros32                       0x08001d2d   Thumb Code    18  cpu_core.o(.text)
    CPU_CntLeadZeros64                       0x08001d3f   Thumb Code   188  cpu_core.o(.text)
    CPU_CntTrailZeros08                      0x08001dfb   Thumb Code    22  cpu_core.o(.text)
    CPU_CntTrailZeros16                      0x08001e11   Thumb Code    22  cpu_core.o(.text)
    CPU_CntTrailZeros32                      0x08001e27   Thumb Code    22  cpu_core.o(.text)
    CPU_CntTrailZeros64                      0x08001e3d   Thumb Code    62  cpu_core.o(.text)
    CPU_IntDis                               0x08001e89   Thumb Code     0  cpu_a.o(.text)
    CPU_IntEn                                0x08001e8d   Thumb Code     0  cpu_a.o(.text)
    CPU_SR_Save                              0x08001e91   Thumb Code     0  cpu_a.o(.text)
    CPU_SR_Restore                           0x08001e99   Thumb Code     0  cpu_a.o(.text)
    CPU_WaitForInt                           0x08001e9f   Thumb Code     0  cpu_a.o(.text)
    CPU_WaitForExcept                        0x08001ea3   Thumb Code     0  cpu_a.o(.text)
    CPU_CntLeadZeros                         0x08001ea7   Thumb Code     0  cpu_a.o(.text)
    CPU_CntTrailZeros                        0x08001ead   Thumb Code     0  cpu_a.o(.text)
    CPU_RevBits                              0x08001eb7   Thumb Code     0  cpu_a.o(.text)
    CPU_BitBandClr                           0x08001ebd   Thumb Code    58  cpu_c.o(.text)
    CPU_BitBandSet                           0x08001ef7   Thumb Code    58  cpu_c.o(.text)
    CPU_IntSrcDis                            0x08001f31   Thumb Code   328  cpu_c.o(.text)
    CPU_IntSrcEn                             0x08002079   Thumb Code   328  cpu_c.o(.text)
    CPU_IntSrcPendClr                        0x080021c1   Thumb Code   164  cpu_c.o(.text)
    CPU_IntSrcPrioSet                        0x08002265   Thumb Code   522  cpu_c.o(.text)
    CPU_IntSrcPrioGet                        0x0800246f   Thumb Code   450  cpu_c.o(.text)
    ASCII_IsAlpha                            0x08002639   Thumb Code    48  lib_ascii.o(.text)
    ASCII_IsAlphaNum                         0x08002669   Thumb Code    76  lib_ascii.o(.text)
    ASCII_IsLower                            0x080026b5   Thumb Code    20  lib_ascii.o(.text)
    ASCII_IsUpper                            0x080026c9   Thumb Code    20  lib_ascii.o(.text)
    ASCII_IsDig                              0x080026dd   Thumb Code    20  lib_ascii.o(.text)
    ASCII_IsDigOct                           0x080026f1   Thumb Code    20  lib_ascii.o(.text)
    ASCII_IsDigHex                           0x08002705   Thumb Code    36  lib_ascii.o(.text)
    ASCII_IsBlank                            0x08002729   Thumb Code    20  lib_ascii.o(.text)
    ASCII_IsSpace                            0x0800273d   Thumb Code    36  lib_ascii.o(.text)
    ASCII_IsPrint                            0x08002761   Thumb Code    20  lib_ascii.o(.text)
    ASCII_IsGraph                            0x08002775   Thumb Code    20  lib_ascii.o(.text)
    ASCII_IsPunct                            0x08002789   Thumb Code   134  lib_ascii.o(.text)
    ASCII_IsCtrl                             0x0800280f   Thumb Code    26  lib_ascii.o(.text)
    ASCII_ToLower                            0x08002829   Thumb Code    32  lib_ascii.o(.text)
    ASCII_ToUpper                            0x08002849   Thumb Code    32  lib_ascii.o(.text)
    ASCII_Cmp                                0x08002869   Thumb Code    38  lib_ascii.o(.text)
    Mem_Init                                 0x08002891   Thumb Code    54  lib_mem.o(.text)
    Mem_Set                                  0x080028c7   Thumb Code    98  lib_mem.o(.text)
    Mem_Clr                                  0x08002929   Thumb Code    18  lib_mem.o(.text)
    Mem_Move                                 0x0800293b   Thumb Code   204  lib_mem.o(.text)
    Mem_Cmp                                  0x08002a07   Thumb Code   192  lib_mem.o(.text)
    Mem_HeapAlloc                            0x08002bbb   Thumb Code   256  lib_mem.o(.text)
    Mem_SegGetSizeRem                        0x08002cbb   Thumb Code   214  lib_mem.o(.text)
    Mem_HeapGetSizeRem                       0x08002d91   Thumb Code    22  lib_mem.o(.text)
    Mem_PoolClr                              0x08002da7   Thumb Code    78  lib_mem.o(.text)
    Mem_PoolCreate                           0x08002df5   Thumb Code  1076  lib_mem.o(.text)
    Mem_PoolBlkGetNbrAvail                   0x08003229   Thumb Code   128  lib_mem.o(.text)
    Mem_PoolBlkGet                           0x080032a9   Thumb Code   224  lib_mem.o(.text)
    Mem_PoolBlkGetUsedAtIx                   0x08003389   Thumb Code   212  lib_mem.o(.text)
    Mem_PoolBlkFree                          0x080034c3   Thumb Code   338  lib_mem.o(.text)
    Mem_PoolBlkIxGet                         0x08003615   Thumb Code   314  lib_mem.o(.text)
    Str_Len_N                                0x08003755   Thumb Code    28  lib_str.o(.text)
    Str_Len                                  0x08003771   Thumb Code    20  lib_str.o(.text)
    Str_Copy_N                               0x08003785   Thumb Code    70  lib_str.o(.text)
    Str_Copy                                 0x080037cb   Thumb Code    24  lib_str.o(.text)
    Str_Cat_N                                0x080037e3   Thumb Code    90  lib_str.o(.text)
    Str_Cat                                  0x0800383d   Thumb Code    24  lib_str.o(.text)
    Str_Cmp_N                                0x08003855   Thumb Code   156  lib_str.o(.text)
    Str_Cmp                                  0x080038f1   Thumb Code    24  lib_str.o(.text)
    Str_CmpIgnoreCase_N                      0x08003909   Thumb Code   264  lib_str.o(.text)
    Str_CmpIgnoreCase                        0x08003a11   Thumb Code    24  lib_str.o(.text)
    Str_Char_N                               0x08003a29   Thumb Code    74  lib_str.o(.text)
    Str_Char                                 0x08003a73   Thumb Code    24  lib_str.o(.text)
    Str_Char_Last_N                          0x08003a8b   Thumb Code    76  lib_str.o(.text)
    Str_Char_Last                            0x08003ad7   Thumb Code    24  lib_str.o(.text)
    Str_Char_Replace_N                       0x08003aef   Thumb Code    52  lib_str.o(.text)
    Str_Char_Replace                         0x08003b23   Thumb Code    28  lib_str.o(.text)
    Str_Str_N                                0x08003b3f   Thumb Code   182  lib_str.o(.text)
    Str_Str                                  0x08003bf5   Thumb Code    24  lib_str.o(.text)
    Str_FmtNbr_Int32U                        0x08003de7   Thumb Code    46  lib_str.o(.text)
    Str_FmtNbr_Int32S                        0x08003e15   Thumb Code    62  lib_str.o(.text)
    Str_ParseNbr_Int32U                      0x08004011   Thumb Code    30  lib_str.o(.text)
    Str_ParseNbr_Int32S                      0x0800402f   Thumb Code    74  lib_str.o(.text)
    Mem_Copy                                 0x0800407d   Thumb Code     0  lib_mem_a.o(.text)
    OSCfg_Init                               0x0800429d   Thumb Code     2  os_cfg_app.o(.text)
    OS_IdleTask                              0x080042a1   Thumb Code    50  os_core.o(.text)
    OS_IdleTaskInit                          0x080042d3   Thumb Code    68  os_core.o(.text)
    OS_RdyListInit                           0x08004317   Thumb Code    32  os_core.o(.text)
    OSInit                                   0x08004337   Thumb Code   276  os_core.o(.text)
    OSIntEnter                               0x0800444b   Thumb Code    34  os_core.o(.text)
    OSIntExit                                0x0800446d   Thumb Code   188  os_core.o(.text)
    OSSched                                  0x08004529   Thumb Code   130  os_core.o(.text)
    OS_SchedLockTimeMeasStart                0x080045ab   Thumb Code    20  os_core.o(.text)
    OSSchedLock                              0x080045bf   Thumb Code   104  os_core.o(.text)
    OS_SchedLockTimeMeasStop                 0x08004627   Thumb Code    44  os_core.o(.text)
    OSSchedUnlock                            0x08004653   Thumb Code   284  os_core.o(.text)
    OSSchedRoundRobinCfg                     0x0800476f   Thumb Code    88  os_core.o(.text)
    OS_RdyListMoveHeadToTail                 0x080047c7   Thumb Code    68  os_core.o(.text)
    OSSchedRoundRobinYield                   0x0800480b   Thumb Code   164  os_core.o(.text)
    OSStart                                  0x080048af   Thumb Code    78  os_core.o(.text)
    OSVersion                                0x080048fd   Thumb Code    12  os_core.o(.text)
    OS_PendDbgNameAdd                        0x08004909   Thumb Code    66  os_core.o(.text)
    OS_PendListInsertPrio                    0x0800494b   Thumb Code   102  os_core.o(.text)
    OS_PendDataInit                          0x080049b1   Thumb Code    38  os_core.o(.text)
    OS_RdyListRemove                         0x080049d7   Thumb Code    86  os_core.o(.text)
    OS_TaskBlock                             0x08004a2d   Thumb Code    56  os_core.o(.text)
    OS_Pend                                  0x08004a65   Thumb Code    98  os_core.o(.text)
    OS_PendListRemove1                       0x08004ac7   Thumb Code    66  os_core.o(.text)
    OS_PendListRemove                        0x08004b09   Thumb Code    48  os_core.o(.text)
    OS_PendAbort1                            0x08004b39   Thumb Code    36  os_core.o(.text)
    OS_RdyListInsertHead                     0x08004b5d   Thumb Code   128  os_core.o(.text)
    OS_RdyListInsertTail                     0x08004bdd   Thumb Code    56  os_core.o(.text)
    OS_RdyListInsert                         0x08004c15   Thumb Code    40  os_core.o(.text)
    OS_TaskRdy                               0x08004c3d   Thumb Code    28  os_core.o(.text)
    OS_PendAbort                             0x08004c59   Thumb Code   166  os_core.o(.text)
    OS_PendDbgNameRemove                     0x08004cff   Thumb Code    34  os_core.o(.text)
    OS_PendListChangePrio                    0x08004d21   Thumb Code    70  os_core.o(.text)
    OS_PendListInit                          0x08004d67   Thumb Code    10  os_core.o(.text)
    OS_PendListInsertHead                    0x08004d71   Thumb Code    32  os_core.o(.text)
    OS_PendObjDel1                           0x08004d91   Thumb Code    36  os_core.o(.text)
    OS_PendObjDel                            0x08004db5   Thumb Code   162  os_core.o(.text)
    OS_Post1                                 0x08004e57   Thumb Code    42  os_core.o(.text)
    OS_Post                                  0x08004e81   Thumb Code   192  os_core.o(.text)
    OS_SchedRoundRobin                       0x08004f41   Thumb Code   210  os_core.o(.text)
    OS_Dbg_Init                              0x08005019   Thumb Code   148  os_dbg.o(.text)
    OS_FlagDbgListAdd                        0x080051c5   Thumb Code    38  os_flag.o(.text)
    OSFlagCreate                             0x080051eb   Thumb Code   116  os_flag.o(.text)
    OS_FlagBlock                             0x0800525f   Thumb Code    58  os_flag.o(.text)
    OSFlagPend                               0x08005299   Thumb Code   902  os_flag.o(.text)
    OSFlagPendGetFlagsRdy                    0x0800561f   Thumb Code    68  os_flag.o(.text)
    OS_FlagTaskRdy                           0x08005663   Thumb Code    86  os_flag.o(.text)
    OS_FlagPost                              0x080056b9   Thumb Code   350  os_flag.o(.text)
    OSFlagPost                               0x08005817   Thumb Code   112  os_flag.o(.text)
    OS_FlagClr                               0x08005887   Thumb Code    28  os_flag.o(.text)
    OS_FlagInit                              0x080058a3   Thumb Code    14  os_flag.o(.text)
    OS_FlagDbgListRemove                     0x080058b1   Thumb Code    44  os_flag.o(.text)
    OS_MemDbgListAdd                         0x080058fd   Thumb Code    34  os_mem.o(.text)
    OSMemCreate                              0x0800591f   Thumb Code   232  os_mem.o(.text)
    OSMemGet                                 0x08005a07   Thumb Code   100  os_mem.o(.text)
    OSMemPut                                 0x08005a6b   Thumb Code   112  os_mem.o(.text)
    OS_MemInit                               0x08005adb   Thumb Code    14  os_mem.o(.text)
    OS_MsgPoolInit                           0x08005af9   Thumb Code   110  os_msg.o(.text)
    OS_MsgQFreeAll                           0x08005b67   Thumb Code    62  os_msg.o(.text)
    OS_MsgQInit                              0x08005ba5   Thumb Code    14  os_msg.o(.text)
    OS_MsgQGet                               0x08005bb3   Thumb Code    98  os_msg.o(.text)
    OS_MsgQPut                               0x08005c15   Thumb Code   254  os_msg.o(.text)
    OS_MutexDbgListAdd                       0x08005d21   Thumb Code    38  os_mutex.o(.text)
    OSMutexCreate                            0x08005d47   Thumb Code   122  os_mutex.o(.text)
    OSMutexPend                              0x08005dc1   Thumb Code   574  os_mutex.o(.text)
    OSMutexPost                              0x08005fff   Thumb Code   388  os_mutex.o(.text)
    OS_MutexClr                              0x08006183   Thumb Code    38  os_mutex.o(.text)
    OS_MutexDbgListRemove                    0x080061a9   Thumb Code    44  os_mutex.o(.text)
    OS_MutexInit                             0x080061d5   Thumb Code    14  os_mutex.o(.text)
    OS_PrioInit                              0x080061f9   Thumb Code    20  os_prio.o(.text)
    OS_PrioGetHighest                        0x0800620d   Thumb Code    36  os_prio.o(.text)
    OS_PrioInsert                            0x08006231   Thumb Code    32  os_prio.o(.text)
    OS_PrioRemove                            0x08006251   Thumb Code    32  os_prio.o(.text)
    OS_QDbgListAdd                           0x08006275   Thumb Code    38  os_q.o(.text)
    OSQCreate                                0x0800629b   Thumb Code   130  os_q.o(.text)
    OSQPend                                  0x0800631d   Thumb Code   446  os_q.o(.text)
    OSQPendAbort                             0x080064db   Thumb Code   236  os_q.o(.text)
    OS_QPost                                 0x080065c7   Thumb Code   220  os_q.o(.text)
    OSQPost                                  0x080066a3   Thumb Code   144  os_q.o(.text)
    OS_QClr                                  0x08006733   Thumb Code    40  os_q.o(.text)
    OS_QDbgListRemove                        0x0800675b   Thumb Code    44  os_q.o(.text)
    OS_QInit                                 0x08006787   Thumb Code    14  os_q.o(.text)
    OS_SemDbgListAdd                         0x080067a9   Thumb Code    38  os_sem.o(.text)
    OSSemCreate                              0x080067cf   Thumb Code   116  os_sem.o(.text)
    OSSemPend                                0x08006843   Thumb Code   406  os_sem.o(.text)
    OSSemPendAbort                           0x080069d9   Thumb Code   236  os_sem.o(.text)
    OS_SemPost                               0x08006ac5   Thumb Code   322  os_sem.o(.text)
    OSSemPost                                0x08006c07   Thumb Code   108  os_sem.o(.text)
    OSSemSet                                 0x08006c73   Thumb Code   120  os_sem.o(.text)
    OS_SemClr                                0x08006ceb   Thumb Code    28  os_sem.o(.text)
    OS_SemDbgListRemove                      0x08006d07   Thumb Code    44  os_sem.o(.text)
    OS_SemInit                               0x08006d33   Thumb Code    14  os_sem.o(.text)
    OSTaskChangePrio                         0x08006d5d   Thumb Code   274  os_task.o(.text)
    OS_TaskDbgListAdd                        0x08006e6f   Thumb Code    42  os_task.o(.text)
    OS_TaskInitTCB                           0x08006e99   Thumb Code   190  os_task.o(.text)
    OSTaskCreate                             0x08006f57   Thumb Code   412  os_task.o(.text)
    OS_TaskDbgListRemove                     0x080070f3   Thumb Code    64  os_task.o(.text)
    OSTaskDel                                0x08007133   Thumb Code   324  os_task.o(.text)
    OSTaskQFlush                             0x08007277   Thumb Code   110  os_task.o(.text)
    OSTaskQPend                              0x080072e5   Thumb Code   458  os_task.o(.text)
    OS_TaskQPost                             0x080074af   Thumb Code   242  os_task.o(.text)
    OSTaskQPost                              0x080075a1   Thumb Code    82  os_task.o(.text)
    OSTaskRegGet                             0x080075f3   Thumb Code    78  os_task.o(.text)
    OSTaskRegGetID                           0x08007641   Thumb Code    84  os_task.o(.text)
    OSTaskRegSet                             0x08007695   Thumb Code    78  os_task.o(.text)
    OS_TaskResume                            0x080076e3   Thumb Code   256  os_task.o(.text)
    OSTaskResume                             0x080077e3   Thumb Code    96  os_task.o(.text)
    OSTaskSemPend                            0x08007843   Thumb Code   482  os_task.o(.text)
    OSTaskSemPendAbort                       0x08007a25   Thumb Code   214  os_task.o(.text)
    OS_TaskSemPost                           0x08007afb   Thumb Code   448  os_task.o(.text)
    OSTaskSemPost                            0x08007cbb   Thumb Code    62  os_task.o(.text)
    OSTaskSemSet                             0x08007cf9   Thumb Code    80  os_task.o(.text)
    OSTaskStkChk                             0x08007d49   Thumb Code   212  os_task.o(.text)
    OS_TaskSuspend                           0x08007e1d   Thumb Code   272  os_task.o(.text)
    OSTaskSuspend                            0x08007f2d   Thumb Code    48  os_task.o(.text)
    OSTaskTimeQuantaSet                      0x08007f5d   Thumb Code    96  os_task.o(.text)
    OS_TaskInit                              0x08007fbd   Thumb Code    18  os_task.o(.text)
    OS_TaskReturn                            0x08007fcf   Thumb Code    20  os_task.o(.text)
    OS_TickListRemove                        0x08008005   Thumb Code    56  os_tick.o(.text)
    OS_TickListUpdate                        0x0800803d   Thumb Code   376  os_tick.o(.text)
    OS_TickTask                              0x080081b5   Thumb Code    38  os_tick.o(.text)
    OS_TickListInit                          0x080081db   Thumb Code    32  os_tick.o(.text)
    OS_TickTaskInit                          0x080081fb   Thumb Code   130  os_tick.o(.text)
    OS_TickListInsert                        0x0800827d   Thumb Code   430  os_tick.o(.text)
    OS_TickListResetPeak                     0x0800842b   Thumb Code    94  os_tick.o(.text)
    OSTimeDly                                0x08008489   Thumb Code   182  os_time.o(.text)
    OSTimeDlyHMSM                            0x0800853f   Thumb Code   394  os_time.o(.text)
    OSTimeGet                                0x080086c9   Thumb Code    46  os_time.o(.text)
    OSTimeSet                                0x080086f7   Thumb Code    46  os_time.o(.text)
    OSTimeTick                               0x08008725   Thumb Code    68  os_time.o(.text)
    OS_TmrDbgListAdd                         0x08008795   Thumb Code    34  os_tmr.o(.text)
    OSTmrCreate                              0x080087b7   Thumb Code   192  os_tmr.o(.text)
    OSTmrRemainGet                           0x08008877   Thumb Code   188  os_tmr.o(.text)
    OS_TmrLink                               0x08008933   Thumb Code   196  os_tmr.o(.text)
    OS_TmrUnlink                             0x080089f7   Thumb Code    72  os_tmr.o(.text)
    OSTmrStart                               0x08008a3f   Thumb Code   170  os_tmr.o(.text)
    OSTmrStateGet                            0x08008ae9   Thumb Code   134  os_tmr.o(.text)
    OSTmrStop                                0x08008b6f   Thumb Code   276  os_tmr.o(.text)
    OS_TmrClr                                0x08008c83   Thumb Code    36  os_tmr.o(.text)
    OS_TmrDbgListRemove                      0x08008ca7   Thumb Code    44  os_tmr.o(.text)
    OS_TmrTask                               0x08008cd3   Thumb Code   176  os_tmr.o(.text)
    OS_TmrInit                               0x08008d83   Thumb Code   208  os_tmr.o(.text)
    OS_TmrResetPeak                          0x08008e53   Thumb Code    28  os_tmr.o(.text)
    OSIdleTaskHook                           0x08008ed5   Thumb Code    16  os_cpu_c.o(.text)
    OSInitHook                               0x08008ee5   Thumb Code    28  os_cpu_c.o(.text)
    OSStatTaskHook                           0x08008f01   Thumb Code    16  os_cpu_c.o(.text)
    OSTaskCreateHook                         0x08008f11   Thumb Code    20  os_cpu_c.o(.text)
    OSTaskDelHook                            0x08008f25   Thumb Code    20  os_cpu_c.o(.text)
    OSTaskReturnHook                         0x08008f39   Thumb Code    20  os_cpu_c.o(.text)
    OSTaskStkInit                            0x08008f4d   Thumb Code   192  os_cpu_c.o(.text)
    OSTaskSwHook                             0x0800900d   Thumb Code   120  os_cpu_c.o(.text)
    OSTimeTickHook                           0x08009085   Thumb Code    16  os_cpu_c.o(.text)
    OS_CPU_SysTickHandler                    0x08009095   Thumb Code    52  os_cpu_c.o(.text)
    OS_CPU_SysTickInit                       0x080090c9   Thumb Code    44  os_cpu_c.o(.text)
    __aeabi_uldivmod                         0x08009135   Thumb Code    98  uldiv.o(.text)
    __aeabi_llsl                             0x08009197   Thumb Code    30  llshl.o(.text)
    _ll_shift_l                              0x08009197   Thumb Code     0  llshl.o(.text)
    __aeabi_llsr                             0x080091b5   Thumb Code    32  llushr.o(.text)
    _ll_ushift_r                             0x080091b5   Thumb Code     0  llushr.o(.text)
    __scatterload                            0x080091d5   Thumb Code    28  init.o(.text)
    __scatterload_rt2                        0x080091d5   Thumb Code     0  init.o(.text)
    OSStartHighRdy                           0x080091f9   Thumb Code     0  os_cpu_a.o(CODE)
    OSCtxSw                                  0x0800921b   Thumb Code     0  os_cpu_a.o(CODE)
    OSIntCtxSw                               0x08009225   Thumb Code     0  os_cpu_a.o(CODE)
    OS_CPU_PendSVHandler                     0x0800922f   Thumb Code     0  os_cpu_a.o(CODE)
    __scatterload_copy                       0x08009291   Thumb Code    14  handlers.o(i.__scatterload_copy)
    __scatterload_null                       0x0800929f   Thumb Code     2  handlers.o(i.__scatterload_null)
    __scatterload_zeroinit                   0x080092a1   Thumb Code    14  handlers.o(i.__scatterload_zeroinit)
    OSCfg_IdleTaskStkBasePtr                 0x08009444   Data           4  os_cfg_app.o(.constdata)
    OSCfg_IdleTaskStkLimit                   0x08009448   Data           4  os_cfg_app.o(.constdata)
    OSCfg_IdleTaskStkSize                    0x0800944c   Data           4  os_cfg_app.o(.constdata)
    OSCfg_IdleTaskStkSizeRAM                 0x08009450   Data           4  os_cfg_app.o(.constdata)
    OSCfg_IntQBasePtr                        0x08009454   Data           4  os_cfg_app.o(.constdata)
    OSCfg_IntQSize                           0x08009458   Data           2  os_cfg_app.o(.constdata)
    OSCfg_IntQSizeRAM                        0x0800945c   Data           4  os_cfg_app.o(.constdata)
    OSCfg_IntQTaskStkBasePtr                 0x08009460   Data           4  os_cfg_app.o(.constdata)
    OSCfg_IntQTaskStkLimit                   0x08009464   Data           4  os_cfg_app.o(.constdata)
    OSCfg_IntQTaskStkSize                    0x08009468   Data           4  os_cfg_app.o(.constdata)
    OSCfg_IntQTaskStkSizeRAM                 0x0800946c   Data           4  os_cfg_app.o(.constdata)
    OSCfg_ISRStkBasePtr                      0x08009470   Data           4  os_cfg_app.o(.constdata)
    OSCfg_ISRStkSize                         0x08009474   Data           4  os_cfg_app.o(.constdata)
    OSCfg_ISRStkSizeRAM                      0x08009478   Data           4  os_cfg_app.o(.constdata)
    OSCfg_MsgPoolSize                        0x0800947c   Data           2  os_cfg_app.o(.constdata)
    OSCfg_MsgPoolSizeRAM                     0x08009480   Data           4  os_cfg_app.o(.constdata)
    OSCfg_MsgPoolBasePtr                     0x08009484   Data           4  os_cfg_app.o(.constdata)
    OSCfg_StatTaskPrio                       0x08009488   Data           1  os_cfg_app.o(.constdata)
    OSCfg_StatTaskRate_Hz                    0x0800948c   Data           4  os_cfg_app.o(.constdata)
    OSCfg_StatTaskStkBasePtr                 0x08009490   Data           4  os_cfg_app.o(.constdata)
    OSCfg_StatTaskStkLimit                   0x08009494   Data           4  os_cfg_app.o(.constdata)
    OSCfg_StatTaskStkSize                    0x08009498   Data           4  os_cfg_app.o(.constdata)
    OSCfg_StatTaskStkSizeRAM                 0x0800949c   Data           4  os_cfg_app.o(.constdata)
    OSCfg_StkSizeMin                         0x080094a0   Data           4  os_cfg_app.o(.constdata)
    OSCfg_TickRate_Hz                        0x080094a4   Data           4  os_cfg_app.o(.constdata)
    OSCfg_TickTaskPrio                       0x080094a8   Data           1  os_cfg_app.o(.constdata)
    OSCfg_TickTaskStkBasePtr                 0x080094ac   Data           4  os_cfg_app.o(.constdata)
    OSCfg_TickTaskStkLimit                   0x080094b0   Data           4  os_cfg_app.o(.constdata)
    OSCfg_TickTaskStkSize                    0x080094b4   Data           4  os_cfg_app.o(.constdata)
    OSCfg_TickTaskStkSizeRAM                 0x080094b8   Data           4  os_cfg_app.o(.constdata)
    OSCfg_TickWheelSize                      0x080094bc   Data           2  os_cfg_app.o(.constdata)
    OSCfg_TickWheelSizeRAM                   0x080094c0   Data           4  os_cfg_app.o(.constdata)
    OSCfg_TmrTaskPrio                        0x080094c4   Data           1  os_cfg_app.o(.constdata)
    OSCfg_TmrTaskRate_Hz                     0x080094c8   Data           4  os_cfg_app.o(.constdata)
    OSCfg_TmrTaskStkBasePtr                  0x080094cc   Data           4  os_cfg_app.o(.constdata)
    OSCfg_TmrTaskStkLimit                    0x080094d0   Data           4  os_cfg_app.o(.constdata)
    OSCfg_TmrTaskStkSize                     0x080094d4   Data           4  os_cfg_app.o(.constdata)
    OSCfg_TmrTaskStkSizeRAM                  0x080094d8   Data           4  os_cfg_app.o(.constdata)
    OSCfg_TmrWheelSize                       0x080094dc   Data           2  os_cfg_app.o(.constdata)
    OSCfg_TmrWheelSizeRAM                    0x080094e0   Data           4  os_cfg_app.o(.constdata)
    OSCfg_DataSizeRAM                        0x080094e4   Data           4  os_cfg_app.o(.constdata)
    OSDbg_DbgEn                              0x080094e8   Data           1  os_dbg.o(.constdata)
    OSDbg_ArgChkEn                           0x080094e9   Data           1  os_dbg.o(.constdata)
    OSDbg_AppHooksEn                         0x080094ea   Data           1  os_dbg.o(.constdata)
    OSDbg_EndiannessTest                     0x080094ec   Data           4  os_dbg.o(.constdata)
    OSDbg_CalledFromISRChkEn                 0x080094f0   Data           1  os_dbg.o(.constdata)
    OSDbg_FlagEn                             0x080094f1   Data           1  os_dbg.o(.constdata)
    OSDbg_FlagGrp                            0x080094f4   Data          40  os_dbg.o(.constdata)
    OSDbg_FlagDelEn                          0x0800951c   Data           1  os_dbg.o(.constdata)
    OSDbg_FlagModeClrEn                      0x0800951d   Data           1  os_dbg.o(.constdata)
    OSDbg_FlagPendAbortEn                    0x0800951e   Data           1  os_dbg.o(.constdata)
    OSDbg_FlagGrpSize                        0x08009520   Data           2  os_dbg.o(.constdata)
    OSDbg_FlagWidth                          0x08009522   Data           2  os_dbg.o(.constdata)
    OSDbg_IntQ                               0x08009524   Data           2  os_dbg.o(.constdata)
    OSDbg_ISRPostDeferredEn                  0x08009526   Data           1  os_dbg.o(.constdata)
    OSDbg_Mem                                0x08009528   Data          32  os_dbg.o(.constdata)
    OSDbg_MemEn                              0x08009548   Data           1  os_dbg.o(.constdata)
    OSDbg_MemSize                            0x0800954a   Data           2  os_dbg.o(.constdata)
    OSDbg_MsgEn                              0x0800954c   Data           1  os_dbg.o(.constdata)
    OSDbg_MsgSize                            0x0800954e   Data           2  os_dbg.o(.constdata)
    OSDbg_MsgPoolSize                        0x08009550   Data           2  os_dbg.o(.constdata)
    OSDbg_MsgQSize                           0x08009552   Data           2  os_dbg.o(.constdata)
    OSDbg_Mutex                              0x08009554   Data          44  os_dbg.o(.constdata)
    OSDbg_MutexEn                            0x08009580   Data           1  os_dbg.o(.constdata)
    OSDbg_MutexDelEn                         0x08009581   Data           1  os_dbg.o(.constdata)
    OSDbg_MutexPendAbortEn                   0x08009582   Data           1  os_dbg.o(.constdata)
    OSDbg_MutexSize                          0x08009584   Data           2  os_dbg.o(.constdata)
    OSDbg_ObjTypeChkEn                       0x08009586   Data           1  os_dbg.o(.constdata)
    OSDbg_PendMultiEn                        0x08009587   Data           1  os_dbg.o(.constdata)
    OSDbg_PendDataSize                       0x08009588   Data           2  os_dbg.o(.constdata)
    OSDbg_PendListSize                       0x0800958a   Data           2  os_dbg.o(.constdata)
    OSDbg_PendObjSize                        0x0800958c   Data           2  os_dbg.o(.constdata)
    OSDbg_PrioMax                            0x0800958e   Data           2  os_dbg.o(.constdata)
    OSDbg_PrioTblSize                        0x08009590   Data           2  os_dbg.o(.constdata)
    OSDbg_PtrSize                            0x08009592   Data           2  os_dbg.o(.constdata)
    OSDbg_Q                                  0x08009594   Data          48  os_dbg.o(.constdata)
    OSDbg_QEn                                0x080095c4   Data           1  os_dbg.o(.constdata)
    OSDbg_QDelEn                             0x080095c5   Data           1  os_dbg.o(.constdata)
    OSDbg_QFlushEn                           0x080095c6   Data           1  os_dbg.o(.constdata)
    OSDbg_QPendAbortEn                       0x080095c7   Data           1  os_dbg.o(.constdata)
    OSDbg_QSize                              0x080095c8   Data           2  os_dbg.o(.constdata)
    OSDbg_SchedRoundRobinEn                  0x080095ca   Data           1  os_dbg.o(.constdata)
    OSDbg_Sem                                0x080095cc   Data          40  os_dbg.o(.constdata)
    OSDbg_SemEn                              0x080095f4   Data           1  os_dbg.o(.constdata)
    OSDbg_SemDelEn                           0x080095f5   Data           1  os_dbg.o(.constdata)
    OSDbg_SemPendAbortEn                     0x080095f6   Data           1  os_dbg.o(.constdata)
    OSDbg_SemSetEn                           0x080095f7   Data           1  os_dbg.o(.constdata)
    OSDbg_SemSize                            0x080095f8   Data           2  os_dbg.o(.constdata)
    OSDbg_RdyList                            0x080095fa   Data           2  os_dbg.o(.constdata)
    OSDbg_RdyListSize                        0x080095fc   Data           4  os_dbg.o(.constdata)
    OSDbg_StkWidth                           0x08009600   Data           1  os_dbg.o(.constdata)
    OSDbg_StatTaskEn                         0x08009601   Data           1  os_dbg.o(.constdata)
    OSDbg_StatTaskStkChkEn                   0x08009602   Data           1  os_dbg.o(.constdata)
    OSDbg_TaskChangePrioEn                   0x08009603   Data           1  os_dbg.o(.constdata)
    OSDbg_TaskDelEn                          0x08009604   Data           1  os_dbg.o(.constdata)
    OSDbg_TaskQEn                            0x08009605   Data           1  os_dbg.o(.constdata)
    OSDbg_TaskQPendAbortEn                   0x08009606   Data           1  os_dbg.o(.constdata)
    OSDbg_TaskProfileEn                      0x08009607   Data           1  os_dbg.o(.constdata)
    OSDbg_TaskRegTblSize                     0x08009608   Data           2  os_dbg.o(.constdata)
    OSDbg_TaskSemPendAbortEn                 0x0800960a   Data           1  os_dbg.o(.constdata)
    OSDbg_TaskSuspendEn                      0x0800960b   Data           1  os_dbg.o(.constdata)
    OSDbg_TCBSize                            0x0800960c   Data           2  os_dbg.o(.constdata)
    OSDbg_TickSpokeSize                      0x0800960e   Data           2  os_dbg.o(.constdata)
    OSDbg_TimeDlyHMSMEn                      0x08009610   Data           1  os_dbg.o(.constdata)
    OSDbg_TimeDlyResumeEn                    0x08009611   Data           1  os_dbg.o(.constdata)
    OSDbg_TLS_TblSize                        0x08009612   Data           2  os_dbg.o(.constdata)
    OSDbg_Tmr                                0x08009614   Data          52  os_dbg.o(.constdata)
    OSDbg_TmrEn                              0x08009648   Data           1  os_dbg.o(.constdata)
    OSDbg_TmrDelEn                           0x08009649   Data           1  os_dbg.o(.constdata)
    OSDbg_TmrSize                            0x0800964a   Data           2  os_dbg.o(.constdata)
    OSDbg_TmrSpokeSize                       0x0800964c   Data           2  os_dbg.o(.constdata)
    OSDbg_VersionNbr                         0x0800964e   Data           2  os_dbg.o(.constdata)
    OSDbg_DataSize                           0x08009650   Data           4  os_dbg.o(.constdata)
    Region$$Table$$Base                      0x08009654   Number         0  anon$$obj.o(Region$$Table)
    Region$$Table$$Limit                     0x08009674   Number         0  anon$$obj.o(Region$$Table)
    MyDataBlkPtr                             0x20000000   Data           4  app.o(.data)
    counter                                  0x20000004   Data           1  app.o(.data)
    ucKeyCode                                0x20000005   Data           1  app.o(.data)
    ucTemp                                   0x20000006   Data           1  app.o(.data)
    ret                                      0x20000007   Data           1  bsp_key.o(.data)
    SystemCoreClock                          0x20000018   Data           4  system_stm32f2xx.o(.data)
    AHBPrescTable                            0x2000001c   Data          16  system_stm32f2xx.o(.data)
    CPU_TS_TmrFreq_Hz                        0x2000002c   Data           4  cpu_core.o(.data)
    Mem_PoolTbl                              0x20000030   Data           4  lib_mem.o(.data)
    OSPrioTbl                                0x20000034   Data           4  os_prio.o(.data)
    OS_AppTaskCreateHookPtr                  0x20000038   Data           4  os_var.o(.data)
    OS_AppTaskDelHookPtr                     0x2000003c   Data           4  os_var.o(.data)
    OS_AppTaskReturnHookPtr                  0x20000040   Data           4  os_var.o(.data)
    OS_AppIdleTaskHookPtr                    0x20000044   Data           4  os_var.o(.data)
    OS_AppStatTaskHookPtr                    0x20000048   Data           4  os_var.o(.data)
    OS_AppTaskSwHookPtr                      0x2000004c   Data           4  os_var.o(.data)
    OS_AppTimeTickHookPtr                    0x20000050   Data           4  os_var.o(.data)
    OSIdleTaskCtr                            0x20000054   Data           4  os_var.o(.data)
    OSIntNestingCtr                          0x20000058   Data           1  os_var.o(.data)
    OSRunning                                0x20000059   Data           1  os_var.o(.data)
    OSFlagDbgListPtr                         0x2000005c   Data           4  os_var.o(.data)
    OSFlagQty                                0x20000060   Data           2  os_var.o(.data)
    OSMemDbgListPtr                          0x20000064   Data           4  os_var.o(.data)
    OSMemQty                                 0x20000068   Data           2  os_var.o(.data)
    OSMutexDbgListPtr                        0x2000006c   Data           4  os_var.o(.data)
    OSMutexQty                               0x20000070   Data           2  os_var.o(.data)
    OSPrioCur                                0x20000072   Data           1  os_var.o(.data)
    OSPrioHighRdy                            0x20000073   Data           1  os_var.o(.data)
    OSPrioSaved                              0x20000074   Data           1  os_var.o(.data)
    OSQDbgListPtr                            0x20000078   Data           4  os_var.o(.data)
    OSQQty                                   0x2000007c   Data           2  os_var.o(.data)
    OSSchedLockTimeBegin                     0x20000080   Data           4  os_var.o(.data)
    OSSchedLockTimeMax                       0x20000084   Data           4  os_var.o(.data)
    OSSchedLockTimeMaxCur                    0x20000088   Data           4  os_var.o(.data)
    OSSchedLockNestingCtr                    0x2000008c   Data           1  os_var.o(.data)
    OSSchedRoundRobinDfltTimeQuanta          0x20000090   Data           4  os_var.o(.data)
    OSSchedRoundRobinEn                      0x20000094   Data           1  os_var.o(.data)
    OSSemDbgListPtr                          0x20000098   Data           4  os_var.o(.data)
    OSSemQty                                 0x2000009c   Data           2  os_var.o(.data)
    OSTaskCtxSwCtr                           0x200000a0   Data           4  os_var.o(.data)
    OSTaskDbgListPtr                         0x200000a4   Data           4  os_var.o(.data)
    OSTaskQty                                0x200000a8   Data           2  os_var.o(.data)
    OSTaskRegNextAvailID                     0x200000aa   Data           1  os_var.o(.data)
    OSTickCtr                                0x200000ac   Data           4  os_var.o(.data)
    OSTickTaskTimeMax                        0x200000b0   Data           4  os_var.o(.data)
    OSTmrDbgListPtr                          0x200000b4   Data           4  os_var.o(.data)
    OSTmrQty                                 0x200000b8   Data           2  os_var.o(.data)
    OSTmrTaskTimeMax                         0x200000bc   Data           4  os_var.o(.data)
    OSTmrTickCtr                             0x200000c0   Data           4  os_var.o(.data)
    OSTmrUpdateCnt                           0x200000c4   Data           4  os_var.o(.data)
    OSTmrUpdateCtr                           0x200000c8   Data           4  os_var.o(.data)
    OSTCBCurPtr                              0x200000cc   Data           4  os_var.o(.data)
    OSTCBHighRdyPtr                          0x200000d0   Data           4  os_var.o(.data)
    OS_CPU_ExceptStkBase                     0x200000d4   Data           4  os_cpu_c.o(.data)
    RPM_Q                                    0x20003324   Data          48  app.o(.bss)
    MyPartition                              0x20003354   Data          32  app.o(.bss)
    MyPartitionStorage                       0x20003374   Data        1200  app.o(.bss)
    s_tKey                                   0x20003844   Data          13  bsp_key.o(.bss)
    CPU_Name                                 0x20003998   Data          16  cpu_core.o(.bss)
    Mem_PoolHeap                             0x200039a8   Data          72  lib_mem.o(.bss)
    Mem_Heap                                 0x200039f0   Data        9216  lib_mem.o(.bss)
    OSCfg_IdleTaskStk                        0x20005df0   Data         512  os_cfg_app.o(.bss)
    OSCfg_ISRStk                             0x20005ff0   Data        1024  os_cfg_app.o(.bss)
    OSCfg_MsgPool                            0x200063f0   Data         800  os_cfg_app.o(.bss)
    OSCfg_TickTaskStk                        0x20006710   Data         512  os_cfg_app.o(.bss)
    OSCfg_TickWheel                          0x20006910   Data         128  os_cfg_app.o(.bss)
    OSCfg_TmrTaskStk                         0x20006990   Data         512  os_cfg_app.o(.bss)
    OSCfg_TmrWheel                           0x20006b90   Data         128  os_cfg_app.o(.bss)
    OSIdleTaskTCB                            0x20006c10   Data         196  os_var.o(.bss)
    OSMsgPool                                0x20006cd4   Data          12  os_var.o(.bss)
    OSRdyList                                0x20006ce0   Data         144  os_var.o(.bss)
    OSTickTaskTCB                            0x20006d70   Data         196  os_var.o(.bss)
    OSTmrTaskTCB                             0x20006e34   Data         196  os_var.o(.bss)
    __initial_sp                             0x200072f8   Data           0  startup_stm32f2xx.o(STACK)



==============================================================================

Memory Map of the image

  Image Entry point : 0x08000185

  Load Region LR_IROM1 (Base: 0x08000000, Size: 0x0000974c, Max: 0x00100000, ABSOLUTE)

    Execution Region ER_IROM1 (Base: 0x08000000, Size: 0x00009674, Max: 0x00100000, ABSOLUTE)

    Base Addr    Size         Type   Attr      Idx    E Section Name        Object

    0x08000000   0x00000184   Data   RO          281    RESET               startup_stm32f2xx.o
    0x08000184   0x00000000   Code   RO          834  * .ARM.Collect$$$$00000000  mc_w.l(entry.o)
    0x08000184   0x00000004   Code   RO          839    .ARM.Collect$$$$00000001  mc_w.l(entry2.o)
    0x08000188   0x00000004   Code   RO          842    .ARM.Collect$$$$00000004  mc_w.l(entry5.o)
    0x0800018c   0x00000000   Code   RO          844    .ARM.Collect$$$$00000008  mc_w.l(entry7b.o)
    0x0800018c   0x00000000   Code   RO          846    .ARM.Collect$$$$0000000A  mc_w.l(entry8b.o)
    0x0800018c   0x00000008   Code   RO          847    .ARM.Collect$$$$0000000B  mc_w.l(entry9a.o)
    0x08000194   0x00000000   Code   RO          849    .ARM.Collect$$$$0000000D  mc_w.l(entry10a.o)
    0x08000194   0x00000000   Code   RO          851    .ARM.Collect$$$$0000000F  mc_w.l(entry11a.o)
    0x08000194   0x00000004   Code   RO          840    .ARM.Collect$$$$00002712  mc_w.l(entry2.o)
    0x08000198   0x00000260   Code   RO            1    .text               app.o
    0x080003f8   0x000000c8   Code   RO          206    .text               bsp.o
    0x080004c0   0x00000178   Code   RO          218    .text               bsp_led.o
    0x08000638   0x0000004c   Code   RO          234    .text               stm32f2xx_it.o
    0x08000684   0x0000025c   Code   RO          249    .text               bsp_key.o
    0x080008e0   0x0000041c   Code   RO          265    .text               bsp_int.o
    0x08000cfc   0x00000024   Code   RO          282    .text               startup_stm32f2xx.o
    0x08000d20   0x000000e0   Code   RO          287    .text               misc.o
    0x08000e00   0x0000025c   Code   RO          359    .text               stm32f2xx_gpio.o
    0x0800105c   0x00000588   Code   RO          383    .text               stm32f2xx_rcc.o
    0x080015e4   0x0000041a   Code   RO          409    .text               stm32f2xx_usart.o
    0x080019fe   0x00000002   PAD
    0x08001a00   0x000001e0   Code   RO          455    .text               system_stm32f2xx.o
    0x08001be0   0x000002a8   Code   RO          473    .text               cpu_core.o
    0x08001e88   0x00000034   Code   RO          499    .text               cpu_a.o
    0x08001ebc   0x0000077c   Code   RO          502    .text               cpu_c.o
    0x08002638   0x00000256   Code   RO          514    .text               lib_ascii.o
    0x0800288e   0x00000002   PAD
    0x08002890   0x00000ec4   Code   RO          547    .text               lib_mem.o
    0x08003754   0x00000928   Code   RO          566    .text               lib_str.o
    0x0800407c   0x00000220   Code   RO          583    .text               lib_mem_a.o
    0x0800429c   0x00000002   Code   RO          586    .text               os_cfg_app.o
    0x0800429e   0x00000002   PAD
    0x080042a0   0x00000d78   Code   RO          609    .text               os_core.o
    0x08005018   0x000001ac   Code   RO          621    .text               os_dbg.o
    0x080051c4   0x00000738   Code   RO          636    .text               os_flag.o
    0x080058fc   0x000001fc   Code   RO          654    .text               os_mem.o
    0x08005af8   0x00000228   Code   RO          666    .text               os_msg.o
    0x08005d20   0x000004d8   Code   RO          678    .text               os_mutex.o
    0x080061f8   0x0000007c   Code   RO          702    .text               os_prio.o
    0x08006274   0x00000534   Code   RO          721    .text               os_q.o
    0x080067a8   0x000005b4   Code   RO          733    .text               os_sem.o
    0x08006d5c   0x000012a8   Code   RO          751    .text               os_task.o
    0x08008004   0x00000484   Code   RO          763    .text               os_tick.o
    0x08008488   0x0000030c   Code   RO          775    .text               os_time.o
    0x08008794   0x00000740   Code   RO          787    .text               os_tmr.o
    0x08008ed4   0x00000260   Code   RO          816    .text               os_cpu_c.o
    0x08009134   0x00000062   Code   RO          837    .text               mc_w.l(uldiv.o)
    0x08009196   0x0000001e   Code   RO          853    .text               mc_w.l(llshl.o)
    0x080091b4   0x00000020   Code   RO          855    .text               mc_w.l(llushr.o)
    0x080091d4   0x00000024   Code   RO          857    .text               mc_w.l(init.o)
    0x080091f8   0x00000098   Code   RO          813    CODE                os_cpu_a.o
    0x08009290   0x0000000e   Code   RO          861    i.__scatterload_copy  mc_w.l(handlers.o)
    0x0800929e   0x00000002   Code   RO          862    i.__scatterload_null  mc_w.l(handlers.o)
    0x080092a0   0x0000000e   Code   RO          863    i.__scatterload_zeroinit  mc_w.l(handlers.o)
    0x080092ae   0x00000100   Data   RO          475    .constdata          cpu_core.o
    0x080093ae   0x00000002   PAD
    0x080093b0   0x00000094   Data   RO          567    .constdata          lib_str.o
    0x08009444   0x000000a4   Data   RO          588    .constdata          os_cfg_app.o
    0x080094e8   0x0000016c   Data   RO          622    .constdata          os_dbg.o
    0x08009654   0x00000020   Data   RO          859    Region$$Table       anon$$obj.o


    Execution Region RW_IRAM1 (Base: 0x20000000, Size: 0x000072f8, Max: 0x00020000, ABSOLUTE)

    Base Addr    Size         Type   Attr      Idx    E Section Name        Object

    0x20000000   0x00000007   Data   RW            3    .data               app.o
    0x20000007   0x00000001   Data   RW          251    .data               bsp_key.o
    0x20000008   0x00000010   Data   RW          384    .data               stm32f2xx_rcc.o
    0x20000018   0x00000014   Data   RW          456    .data               system_stm32f2xx.o
    0x2000002c   0x00000004   Data   RW          476    .data               cpu_core.o
    0x20000030   0x00000004   Data   RW          549    .data               lib_mem.o
    0x20000034   0x00000004   Data   RW          703    .data               os_prio.o
    0x20000038   0x0000009c   Data   RW          800    .data               os_var.o
    0x200000d4   0x00000004   Data   RW          817    .data               os_cpu_c.o
    0x200000d8   0x0000374c   Zero   RW            2    .bss                app.o
    0x20003824   0x0000002d   Zero   RW          250    .bss                bsp_key.o
    0x20003851   0x00000003   PAD
    0x20003854   0x00000144   Zero   RW          266    .bss                bsp_int.o
    0x20003998   0x00000010   Zero   RW          474    .bss                cpu_core.o
    0x200039a8   0x00002448   Zero   RW          548    .bss                lib_mem.o
    0x20005df0   0x00000e20   Zero   RW          587    .bss                os_cfg_app.o
    0x20006c10   0x000002e8   Zero   RW          799    .bss                os_var.o
    0x20006ef8   0x00000400   Zero   RW          279    STACK               startup_stm32f2xx.o


==============================================================================

Image component sizes


      Code (inc. data)   RO Data    RW Data    ZI Data      Debug   Object Name

       608        148          0          7      14156     276163   app.o
       200         18          0          0          0       1863   bsp.o
      1052          8          0          0        324      13450   bsp_int.o
       604         30          0          1         45       3286   bsp_key.o
       376          4          0          0          0       1413   bsp_led.o
        52          0          0          0          0        304   cpu_a.o
      1916        102          0          0          0       3421   cpu_c.o
       680         14        256          4         16      14016   cpu_core.o
       598          0          0          0          0       3660   lib_ascii.o
      3780         62          0          4       9288      24324   lib_mem.o
       544          0          0          0          0        448   lib_mem_a.o
      2344          4        148          0          0      12974   lib_str.o
       224         20          0          0          0       1833   misc.o
         2          0        164          0       3616      18981   os_cfg_app.o
      3448        264          0          0          0      11751   os_core.o
       152         32          0          0          0        368   os_cpu_a.o
       608         64          0          4          0       3485   os_cpu_c.o
       428        280        364          0          0       4681   os_dbg.o
      1848         68          0          0          0       5549   os_flag.o
       508         16          0          0          0       2584   os_mem.o
       552         14          0          0          0       2550   os_msg.o
      1240         62          0          0          0       3362   os_mutex.o
       124          4          0          4          0       1648   os_prio.o
      1332         48          0          0          0       4640   os_q.o
      1460         56          0          0          0       5063   os_sem.o
      4776        192          0          0          0      12113   os_task.o
      1156         74          0          0          0       3113   os_tick.o
       780         44          0          0          0       2521   os_time.o
      1856        132          0          0          0       5941   os_tmr.o
         0          0          0        156        744      17540   os_var.o
        36          8        388          0       1024        900   startup_stm32f2xx.o
       604         36          0          0          0       3929   stm32f2xx_gpio.o
        76          8          0          0          0       1400   stm32f2xx_it.o
      1416         48          0         16          0      10871   stm32f2xx_rcc.o
      1050         26          0          0          0       7640   stm32f2xx_usart.o
       480         40          0         20          0       1839   system_stm32f2xx.o

    ----------------------------------------------------------------------
     36916       1926       1354        216      29216     489624   Object Totals
         0          0         32          0          0          0   (incl. Generated)
         6          0          2          0          3          0   (incl. Padding)

    ----------------------------------------------------------------------

      Code (inc. data)   RO Data    RW Data    ZI Data      Debug   Library Member Name

         0          0          0          0          0          0   entry.o
         0          0          0          0          0          0   entry10a.o
         0          0          0          0          0          0   entry11a.o
         8          4          0          0          0          0   entry2.o
         4          0          0          0          0          0   entry5.o
         0          0          0          0          0          0   entry7b.o
         0          0          0          0          0          0   entry8b.o
         8          4          0          0          0          0   entry9a.o
        30          0          0          0          0          0   handlers.o
        36          8          0          0          0         68   init.o
        30          0          0          0          0         68   llshl.o
        32          0          0          0          0         68   llushr.o
        98          0          0          0          0         92   uldiv.o

    ----------------------------------------------------------------------
       246         16          0          0          0        296   Library Totals
         0          0          0          0          0          0   (incl. Padding)

    ----------------------------------------------------------------------

      Code (inc. data)   RO Data    RW Data    ZI Data      Debug   Library Name

       246         16          0          0          0        296   mc_w.l

    ----------------------------------------------------------------------
       246         16          0          0          0        296   Library Totals

    ----------------------------------------------------------------------

==============================================================================


      Code (inc. data)   RO Data    RW Data    ZI Data      Debug   

     37162       1942       1354        216      29216     486484   Grand Totals
     37162       1942       1354        216      29216     486484   ELF Image Totals
     37162       1942       1354        216          0          0   ROM Totals

==============================================================================

    Total RO  Size (Code + RO Data)                38516 (  37.61kB)
    Total RW  Size (RW Data + ZI Data)             29432 (  28.74kB)
    Total ROM Size (Code + RO Data + RW Data)      38732 (  37.82kB)

==============================================================================

